:020000040800F2
:1000000068F300205D020008013B0008A1350008EC
:10001000FD3A000851070008F155000800000000F3
:100020000000000000000000000000009D0100082A
:10003000DB0B000800000000F9010008CD490008B2
:1000400077020008770200087702000877020008AC
:10005000770200087702000877020008770200089C
:10006000770200087702000877020008770200088C
:10007000B10A00087702000877020008770200083A
:10008000770200087702000877020008770200086C
:100090005507000877020008770200087702000879
:1000A000770200087702000877020008770200084C
:1000B000770200087702000877020008770200083C
:1000C000770200087702000877020008770200082C
:1000D000770200083955000877020008915500089A
:1000E000770200087702000877020008770200080C
:1000F00077020008770200087702000877020008FC
:1001000077020008770200087702000877020008EB
:100110007702000877020008B14A00087702000859
:100120007702000877020008C10A00087702000879
:1001300077020008770200087702000877020008BB
:1001400065070008770200087702000877020008B8
:10015000770200087702000877020008770200089B
:10016000770200087702000877020008770200088B
:1001700077020008770200087702000800000000FC
:100180007702000877020008DFF80CD000F0BCFA14
:1001900000480047B95B000868F300202C4B196841
:1001A0000868B0E8F04F80F30988BFF36F8F4FF015
:1001B000000080F3118870470000000008480068C4
:1001C000006880F308884FF0000080F3148862B65E
:1001D00061B6BFF34F8FBFF36F8F00DF00BF00BF6B
:1001E00008ED00E0DFF80C00016841F470010160E7
:1001F000704700BF88ED00E0EFF30980BFF36F8F19
:10020000134B1A681EF0100F08BF20ED108A20E96A
:10021000F04F106009B44FF0500080F31188BFF325
:100220004F8FBFF36F8F06F0A7FF4FF0000080F3F2
:10023000118809BC19680868B0E8F04F1EF0100F6B
:1002400008BFB0EC108A80F30988BFF36F8F704746
:1002500044000020EFF30580704700000648804707
:1002600006480047FEE7FEE7FEE7FEE7FEE7FEE79B
:10027000FEE7FEE7FEE7FEE79D4A00088901000869
:100280002DE9F05F0546002092469B4688460646CB
:10029000814640241BE0284641464746224600F05E
:1002A000B4F953465A46C01A914110D31146184624
:1002B000224600F09BF92D1A67EB01084F462246B3
:1002C0000120002100F092F917EB00094E41201E99
:1002D000A4F10104DFDC484631462A464346BDE826
:1002E000F09F40EA01039B0703D009E008C9121FF1
:1002F00008C0042AFAD203E011F8013B00F8013BE0
:10030000521EF9D27047D2B201E000F8012B491E0B
:10031000FBD270470022F6E710B513460A460446A2
:100320001946FFF7F0FF204610BD2DE9FE4F80462D
:1003300081EA0300C00F0C46009021F0004123F039
:100340000045B8EB0200A94105D24046214690463F
:100350001C460B46024623F00040104347D0270DB1
:10036000C7F30A00C3F30A510290401A01904028D3
:100370006BDAC3F3130040F4801B0098924620B15F
:100380000023D2EB030A63EB0B0B01985946C0F133
:100390004002504600F02AF906460D46504659469E
:1003A000019A00F042F910EB08006141002487EA4D
:1003B000115284EAE7731A4340D0009A62B3019A5B
:1003C000012A4FEA075215DC001B61EB02014FF0D6
:1003D000004202EA0752CDE90042001C41F58011BB
:1003E00032462B4600F042F903B0BDE8F08F40469C
:1003F0002146F9E7001B61EB0201001C41F5801367
:1004000000185B412018A2F5001747EB030140EAF2
:10041000D570B6196D4111E06D084FEA360645EA10
:10042000C0754FEA0752001B61EB0201001C41F549
:10043000801149084FEA30000019514132462B46DD
:1004400003B0BDE8F04F00F002B90098012240006F
:100450000023D0EB020263EBE073009821464FEAE1
:10046000E074B8EB000061EB0401E9E783F00043BE
:100470005BE781F0004158E72DE9FE4F81EA030474
:1004800004F0004421F0004100944FF0000B23F0F1
:10049000004350EA01045ED052EA03045BD0C3F388
:1004A0000A54C1F30A552C44A4F2F3340194A0FB7E
:1004B0000254C1F3130141F48011C3F3130343F455
:1004C000801301FB024400FB034E840A970A44EAAE
:1004D000815447EA8357A4FB076802958D0A05FB00
:1004E00007854FEA932C04FB0C542705029D4FEA25
:1004F000065847EA1637B5EB08056EEB070C870E72
:10050000920E47EA811742EA8312A7FB0201B6EB7B
:100510000B0164EB00042B0D43EA0C335E1844EB33
:100520001C50DA465146E7FB0201C5F313044FEABB
:100530000B3343EA14534FEA0432019C43EA0603A7
:10054000A4F10C040294009CCDE900B400F08EF8F4
:1005500003B0BDE8F08F00200146F9E70EB5C10FEA
:1005600080EAE0700844CA07002140F233438DE876
:100570000E000A460B4600F079F803B000BD70B5D6
:10058000C1F30A5201F000450024C1F3130140F207
:10059000FF3341F480119A4201DA002070BD40F22D
:1005A00033439A42A2F2334203DC524200F02DF868
:1005B00000E090402C43F1D0404270BD30B5041EA5
:1005C00071F1000404DB4FF00044404264EB010190
:1005D000141E73F1000405DB1C464FF00043524229
:1005E00063EB04038B4208BF824230BD202A04DB48
:1005F000203A00FA02F1002070479140C2F1200336
:1006000020FA03F3194390407047202A04DB203A74
:1006100021FA02F00021704721FA02F3D040C2F122
:1006200020029140084319467047202A06DBCB1769
:10063000203A41FA02F043EAE07306E041FA02F39D
:10064000D040C2F12002914008431946704710B5CE
:10065000141E73F1000408DA401C41F100019218E5
:100660005B411A4301D120F0010010BD2DE9F04D8E
:1006700092469B4611B1B1FA81F202E0B0FA80F2E3
:1006800020329046FFF7B2FF04460F4640EA0A00C8
:1006900041EA0B0153465A46084313D0114653EA28
:1006A000010019D0C8F140025046FFF7AEFF0546E1
:1006B0000E46504659464246FFF798FF084305D07C
:1006C000012004E020463946BDE8F08D00200543B6
:1006D00046EAE0762C4337430A986305E40AA0EB28
:1006E00008000022FD0A44EA47540A3002D50020DF
:1006F0000146E9E7010510196941DDE908450019DE
:100700006941BDE8F04DA2E7064C074D06E0E06800
:1007100040F0010394E8070098471034AC42F6D348
:10072000FFF736FD408100086081000810B5002405
:1007300008E08021054801F019FB642001F008FA67
:10074000601CC4B2042CF4DB10BD00000018024091
:1007500000BFFEE710B5024800F083FC10BD0000AA
:10076000C400002010B5024800F07BFC10BD000062
:10077000EC00002000B58BB001200990002006900D
:10078000059001900290039004900790012008903A
:100790000E200A9001A9154800F0E4FA08B100F013
:1007A0001DFA124800F053FF08B100F017FA0221B9
:1007B0000E4800F016FA08B100F010FA0E2006906C
:1007C00001A90B4800F0CEFA08B100F007FA08487A
:1007D00000F03DFF08B100F001FA0221044800F0EA
:1007E00000FA08B100F0FAF90BB000BDC400002017
:1007F000EC00002070B506460C480088401C0B49F0
:1008000008804FF400710A4801F0B0FA06F0FCFCD1
:10081000054606F0FFFC0446044800884EF66021B9
:10082000884202DB00200149088070BD00000020E2
:1008300000180240F0B585B006460C4617461D4626
:100840005FA103C9CDE903015DA103C9CDE90101A0
:10085000102E03D05C480088102854D15B480078E3
:1008600010B101284ED124E02F208DF80C008DF816
:10087000040000208DF80D008DF8050010208DF883
:1008800010008DF80800082003AB40F2016200213F
:1008900000904F4805F020F9082001AB40F20262B9
:1008A000002100904A4805F017F9012047490870D7
:1008B00028E02B208DF80C008DF8040001208DF825
:1008C0000D008DF8050000208DF810008DF808004F
:1008D0008DF811008DF80900082003AB40F2016289
:1008E000002100903A4805F0F7F8082001AB40F2EB
:1008F000026200210090364805F0EEF800203349EE
:10090000087000BF5AE03348007810B1012854D174
:1009100027E02F208DF80C008DF8040000208DF8C2
:100920000D008DF805002C4800788DF81000264841
:1009300000788DF80800082003AB40F20162002126
:100940000090234805F0C8F8082001AB40F202628D
:10095000002100901E4805F0BFF801201D490870D5
:100960002BE02B208DF80C008DF8040001208DF871
:100970000D008DF80500E0B28DF81000E8B28DF89A
:100980000800200A8DF81100280A8DF809000820B7
:1009900003AB40F20162002100900D4805F09CF885
:1009A000082001AB40F2026200210090084805F0E7
:1009B00093F800200749087000BF00BF05B0F0BDE4
:1009C0002B002000100000002C0000202E00002032
:1009D000EC0000202F0000202A00002000B585B088
:1009E0002FA003C8CDE903012DA103C9CDE9010161
:1009F0002D48007810B101284ED124E02F208DF829
:100A00000C008DF8040000208DF80D008DF8050015
:100A100010208DF810008DF80800082003AB40F27C
:100A2000016200210090214805F056F8082001AB32
:100A300040F20262002100901C4805F04DF80120B0
:100A40001949087028E02B208DF80C008DF804005F
:100A500001208DF80D008DF8050000208DF81000A4
:100A60008DF808008DF811008DF80900082003ABFF
:100A700040F20162002100900C4805F02DF808209A
:100A800001AB40F2026200210090084805F024F812
:100A900000200549087000BF00BF05B000BD000080
:100AA0002B002000100000002E000020EC00002091
:100AB00010B5024800F06CFE10BD0000BC0800201C
:100AC00010B5024800F064FE10BD00005C08002074
:100AD0000146087810381823B0FBF3F20848805C10
:100AE000C865032A05D908686FF30900001D8865E9
:100AF00003E008686FF309008865886D704700009F
:100B0000BC800008014600208A6A8B69CBB932B1EB
:100B1000012A0DD0022A03D0032A10D10EE000BF13
:100B2000CB6A03F08073B3F1807F00D1012007E02E
:100B3000CB6AB3F1C07F00D1012001E000E000BF2B
:100B400034E08B69B3F5005F1AD132B1012A07D0C6
:100B5000022A03D0032A11D10AE000BF01200EE0CF
:100B6000CB6A03F08073B3F1807F00D1012006E0EF
:100B7000CB6AB3F1C07F00D1012000E000BF15E0D7
:100B800032B1012A05D0022A04D0032A0CD103E095
:100B900000BF00BF012008E0CB6A03F08073B3F10F
:100BA000807F00D1012000E000BF00BF704730B55A
:100BB0000468246824F4802405682C600468636059
:100BC0008468402C04D10468A2600468E16003E0FA
:100BD0000468A1600468E26030BD704772B600BF6F
:100BE000FEE710B5024692F82030012B01D0022B0F
:100BF00006D110684069084314686061002010BD88
:100C0000506A40F4802050620120F8E7F0B50446B5
:100C10000D461E4694F8207020688368A86800B9C5
:100C200000E000BF012F01D0022F7CD103F08060D3
:100C300030B903F0006018B903F08050002873D079
:100C4000C3F30161022905D9606A40F400006062C3
:100C50000120F0BD012088403060A86860B9B5F877
:100C600000C0E86840EA4C5C206800F5C07000EB0A
:100C70000110C0F800C00FE0D5E901C040EACC0087
:100C8000D5F80CC040EA0C00D4F800C00CF5C07CCC
:100C90000CEB011CCCF80000D5F810C0206800F562
:100CA000C07000EB0110C0F804C0287D01280ED1EF
:100CB000206800F5C07000EB0110406840F4807CB3
:100CC000206800F5C07000EB0110C0F804C0D079B6
:100CD000000692F806C040EA0C4092F805C040EACF
:100CE0000C2C10794CEA000C206800F5C07000EB69
:100CF0000110C0F80CC0D078000692F802C040EA9B
:100D00000C4092F801C040EA0C2092F800C040EA82
:100D10000C00D4F800C00CF5C07C0CEB011CCCF826
:100D20000800206801E016E00FE000F5C07000EB5D
:100D30000110006840F0010C206800F5C07000EB65
:100D40000110C0F800C0002083E7606A40F4001082
:100D5000606201207DE7606A40F4802060620120CB
:100D600077E70000F0B504460A46216894F8205061
:100D7000012D01D0022D7ED1424901F50071086894
:100D800040F001000860086820F47C5008600868A2
:100D9000566A40EA06200860107D00F01F06012018
:100DA00000FA06F3C8699843C861A1F50071D069DB
:100DB000C8B9D1F80C029843C1F80C02908880B2EF
:100DC000968940EA064601F51070576940F8376089
:100DD000108880B2168940EA064601F510705769FE
:100DE00000EBC7004660D069012819D1D1F80C0288
:100DF0001843C1F80C02908880B2168840EA064673
:100E000001F51070576940F83760908980B21689F3
:100E100040EA064601F51070576900EBC7004660CE
:100E2000906928B9D1F804029843C1F8040204E09B
:100E3000D1F804021843C1F80402106928B9D1F8A6
:100E400014029843C1F8140204E0D1F814021843C4
:100E5000C1F81402106A012804D1D1F81C02184309
:100E6000C1F81C02D1F8000220F00100C1F8000214
:100E70000020F0BDFFE7606A40F48020606201203E
:100E8000F7E7000000640040704710B502460020FC
:100E900092F82030012B01D0022B09D121B914681E
:100EA000E46804F0030003E01468246904F003001C
:100EB00010BD70B5044694F82050012D01D0022DCC
:100EC0007DD151B92068C06800F0030080B9606A24
:100ED00040F400106062012070BD2068006900F0DD
:100EE000030028B9606A40F4001060620120F3E753
:100EF000206800F5D87000EB0110006800F00400D5
:100F00009060906840B9206800F5D87000EB01103F
:100F10000068400D106007E0206800F5D87000EB15
:100F200001100068C0085060206800F5D87000EB20
:100F30000110006800F00200D060206800F5D87051
:100F400000EB0110406800F00F001061206800F510
:100F5000D87000EB0110406800F47F40000A9061F7
:100F6000206800F5D87000EB01104068000C50615B
:100F7000206800F5D87000EB0110806818702068B8
:100F800000F5D87000EB0110806800F47F40000A83
:100F90005870206800F5D87000EB0110806800F4EC
:100FA0007F00000C9870206800F5D87000EB0110ED
:100FB0008068000ED870206800F5D87000E02FE03F
:100FC00000EB0110C0681871206800F5D87000EBC4
:100FD0000110C06800F47F40000A5871206800F5D5
:100FE000D87000EB0110C06800F47F00000C98710D
:100FF000206800F5D87000EB0110C068000ED871B1
:1010000031B92068C06840F020002668F06005E033
:101010002068006940F020002668306100205BE70E
:10102000606A40F480206062012055E7014600209C
:1010300091F82020012A01D0022A11D10B689B6867
:1010400003F0806303B1401C0B689B6803F00063EE
:1010500003B1401C0B689B6803F0805303B1401C34
:1010600070472DE9F05F0446002520684669206836
:10107000D0F80490206887682068D0F80CA0206819
:10108000D0F810B02068D0F8188006F001000028D1
:1010900055D007F00100C0B101202168886007F039
:1010A000020018B1204600F002FB0EE007F0040039
:1010B00010B145F4006508E007F0080010B145F4F0
:1010C000805502E0204600F0F1FA07F48070C8B1C4
:1010D0004FF480702168886007F4007018B12046D2
:1010E00000F0E7FA0EE007F4806010B145F4005517
:1010F00008E007F4006010B145F4804502E02046A6
:1011000000F0D6FA07F48030C8B14FF4803021687F
:10111000886007F4003018B1204600F0CCFA0EE0E9
:1011200007F4802010B145F4004508E007F40020E2
:1011300010B145F4803502E0204600F0BBFA06F01D
:10114000080038B10AF0100020B145F400751020F5
:101150002168C86006F0040040B10AF0080028B118
:1011600008202168C860204600F00EFA06F0020050
:1011700038B12068C06800F0030010B1204600F0CC
:1011800005FA06F0400038B10BF0100020B145F42C
:10119000806510202168086106F0200040B10BF046
:1011A000080028B1082021680861204600F04CFAA8
:1011B00006F0100038B12068006900F0030010B19B
:1011C000204600F042FA06F4003040B109F0100069
:1011D00028B1102021684860204600F037FA06F454
:1011E000803040B109F0080028B10820216848602B
:1011F000204600F061FA06F4004088B309F00400CC
:1012000078B306F4807020B108F0010008B145F011
:10121000010506F4007020B108F0020008B145F0A5
:10122000020506F4806020B108F0040008B145F022
:10123000040506F40060A0B108F0700088B108F061
:101240007000402817D006DC10280BD020280CD0C6
:10125000302819D10CE0502810D0602814D110E0AB
:101260001DE019E045F008050FE045F010050CE021
:1012700045F0200509E045F0400506E045F0800511
:1012800003E045F4807500E000BF00BF206880697E
:1012900020F07000216888610420216848602DB129
:1012A000606A284360622046FFF7EEFDBDE8F09FCC
:1012B00070B504460CB9012070BD94F8200010B937
:1012C000204600F0AFF82068006840F00100216877
:1012D000086000F05BFD05460DE000F057FD401B87
:1012E0000A2808D9606A40F400306062052084F85A
:1012F00020000120E0E72068406800F0010000289D
:10130000EBD02068006820F002002168086000F03F
:101310003DFD05460DE000F039FD401B0A2808D9C7
:10132000606A40F400306062052084F820000120EB
:10133000C2E72068406800F002000028EBD1207E60
:10134000012806D12068006840F08000216808600C
:1013500005E02068006820F0800021680860607E59
:10136000012806D12068006840F04000216808602C
:1013700005E02068006820F0400021680860A07E39
:10138000012806D12068006840F02000216808602C
:1013900005E02068006820F0200021680860E07EF9
:1013A000012806D12068006820F01000216808603C
:1013B00005E02068006840F0100021680860207F88
:1013C000012806D12068006840F008002168086004
:1013D00005E02068006820F0080021680860607F50
:1013E000012806D12068006840F0040021680860E8
:1013F00005E02068006820F0040021680860D4E956
:101400000201084321690843616908436168491E74
:1014100008432168C86100206062012084F8200030
:10142000002049E710B586B00446142101A8FEF754
:1014300071FF4F492068884242D14E480068401CE5
:101440004C4908600846006801280FD100BF002001
:1014500000904948006840F000704749086008461D
:10146000006800F00070009000BF00BF00BF0020C7
:10147000009041481038006840F001003E491039A2
:1014800008600846006800F00100009000BF00BF3F
:101490004FF4C050019002200290002003900320DE
:1014A00004900920059001A9344800F065FB002252
:1014B0000521142000F064FD142000F051FD55E0DA
:1014C0002F492068884251D100BF002000902A484F
:1014D000006840F08060284908600846006800F015
:1014E0008060009000BF00BF22480068401C214976
:1014F00008600846006801280FD100BF0020009056
:101500001D48006840F000701B49086008460068EC
:1015100000F00070009000BF00BF00BF00200090EE
:1015200015481038006840F002001349103908606F
:101530000846006800F00200009000BF00BF4FF4B2
:10154000405001900220029000200390032004905C
:101550000920059001A90B4800F00EFB002205218F
:10156000402000F00DFD402000F0FAFC06B010BD58
:101570000064004014000020403802400000024097
:1015800000680040000402407047000010B596B0AB
:10159000044600200090019000212046FFF775FCD2
:1015A000254920680968884205D114AB0DAA00219D
:1015B0002046FFF77EFC214920680968884238D11F
:1015C0000BAB04AA00212046FFF773FC40F28251C6
:1015D0000498884214D1DDE90B01CDE902019DF8A0
:1015E00008004F2825D19DF80900122821D19DF827
:1015F0000A0021281DD19DF80C001149087018E03F
:1016000040F281510498884213D1DDE90B01CDE904
:1016100000019DF800004F280BD19DF80100122811
:1016200007D19DF80200212803D19DF80400054947
:10163000087016B010BD0000C4000020EC000020AF
:10164000180000201900002070477047704770B5DF
:10165000044694F82000012822D1022084F82000BA
:101660002068006820F001002168086000F08EFB0F
:1016700005460DE000F08AFB401B0A2808D9606A85
:1016800040F400306062052084F82000012070BD25
:101690002068406800F001000028EBD16062F6E7A6
:1016A000606A40F4002060620120F0E770477047F4
:1016B0007047704770477047704770B50446A56D16
:1016C00000F064FB064694F83500022808D080201C
:1016D000606500BF002084F8340000BF012070BDA9
:1016E0002068006820F016002168086020684069C2
:1016F00020F0800021684861206C08B9A06C28B1F6
:101700002068006820F008002168086020680068F0
:1017100020F001002168086010E000F037FB801B1A
:1017200005280BD920206065032084F8350000BF10
:10173000002084F8340000BF0320D0E72068006850
:1017400000F001000028E8D194F85C103F208840A8
:10175000A860012084F8350000BF002084F8340020
:1017600000BF00BFBBE7014691F83500022803D057
:101770008020486501207047052081F83500086801
:10178000006820F001000A6810600020F3E7000004
:10179000F8B50446002000908C4800684FF41651BC
:1017A000B0FBF1F7A56D2E6894F85C100820884016
:1017B000304098B12068006800F0040070B12068E3
:1017C000006820F004002168086094F85C1008208C
:1017D0008840A860606D40F00100606594F85C107E
:1017E00001208840304068B12068406900F08000E6
:1017F00040B194F85C1001208840A860606D40F012
:101800000200606594F85C1004208840304068B1A4
:101810002068006800F0020040B194F85C100420D9
:101820008840A860606D40F00400606594F85C102A
:1018300010208840304078B32068006800F008002D
:1018400050B394F85C1010208840A86020680068AD
:1018500000F4802080B12068006800F4002028B9DE
:10186000206CC8B12046216C884715E0A06C98B167
:101870002046A16C88470FE02068006800F4807063
:1018800028B92068006820F0080021680860206CF2
:1018900010B12046216C884794F85C1020208840C5
:1018A0003040002865D02068006800F01000002853
:1018B0005FD094F85C1020208840A86094F8350030
:1018C000052828D12068006820F0160021680860EB
:1018D0002068406920F0800021684861206C08B9C8
:1018E000A06C28B12068006820F00800216808601A
:1018F00094F85C103F208840A860012084F83500EF
:1019000000BF002084F8340000BF206D10B12046D5
:10191000216D8847F8BD2068006800F4802080B100
:101920002068006800F4002028B9606C10B12046DF
:10193000616C88471DE0E06BD8B12046E16B8847B9
:1019400017E02068006800F4807068B920680068BB
:1019500020F0100021680860012084F8350000BFE5
:10196000002084F8340000BFE06B10B12046E16B2A
:101970008847606D38B3606D00F00100F0B105205C
:1019800084F835002068006820F0010021680860B4
:1019900000BF0098401C0090B84200D905E02068C4
:1019A000006800F001000028F3D100BF012084F896
:1019B000350000BF002084F8340000BFE06C10B197
:1019C0002046E16C884700BFA4E7000040000020EB
:1019D0002DE9F0410446002500F0D8F9074614B976
:1019E0000120BDE8F081606A00B100BF022084F8E8
:1019F000350000BF002084F8340000BF2068006874
:101A000020F00100216808600AE000F0BFF9C01B67
:101A1000052805D920206065032084F83500E0E71B
:101A20002068006800F001000028EED120680568F9
:101A300021480540D4E901010843E16808432169D0
:101A4000084361690843A1690843E1690843216AC1
:101A500008430543606A042803D1D4E90B01084315
:101A60000543206805602068456925F00705606A20
:101A70000543606A04280DD1A06A0543E06A48B1B5
:101A80002046FFF73FF828B140206065012084F828
:101A90003500A6E7206845612046FFF719F806469D
:101AA00094F85C103F208840B06000206065012001
:101AB00084F83500002094E73F8010F02DE9F047CE
:101AC00004460D4616461F464FF00008D4F85890BD
:101AD00000BF94F83400012802D10220BDE8F0874D
:101AE000012084F8340000BF94F83500012825D186
:101AF000022084F83500002060653B4632462946C6
:101B00002046FFF754F894F85C103F208840C9F84D
:101B100008002068006840F0160021680860206C0A
:101B200028B12068006840F008002168086020683B
:101B3000006840F001002168086006E000BF002056
:101B400084F8340000BF4FF002084046C6E70000AA
:101B500070B5044600F01AF906462546681C10B117
:101B600004480078054400BF00F010F9801BA8422B
:101B7000FAD370BD3C000020F8B502460B460025A4
:101B8000002400200021D6E0012606FA01F51E6897
:101B900006EA0504AC4274D11E7906F00306012E54
:101BA00004D01E7906F00306022E13D190684F0070
:101BB0000326BE40B0434F00DE68BE403043906015
:101BC000506801268E40B0431E79C6F300168E4041
:101BD000304350601E7906F00306032E09D0D0680A
:101BE0004F000326BE40B0434F009E68BE403043C6
:101BF000D0601E7906F00306022E13D1CF0802F141
:101C0000200656F827004E07F70E0F26BE40B043B9
:101C10004F07FF0E1E69BE403043CF0802F1200679
:101C200046F8270010684F000326BE40B0431E79D7
:101C300006F003064F00BE40304310605E6806F4B5
:101C40004036002E76D000BF002600963C4E366807
:101C500046F480463A4F3E603E46366806F480467B
:101C6000009600BF00BF374E8F0856F827008E073A
:101C7000370F0F26BE40B043334EB24202D100268A
:101C800024E057E0314EB24201D101261EE0304E31
:101C9000B24201D1022619E02E4EB24201D10326F2
:101CA00014E02D4EB24201D104260FE02B4EB24279
:101CB00001D105260AE02A4EB24201D1062605E0EE
:101CC000284EB24201D1072600E008268F073F0FB9
:101CD000BE4030431B4E8F0846F82700224E306826
:101CE000A0435E6806F4801606B120431E4E3060A5
:101CF000361D3068A0435E6806F4001606B1204326
:101D0000194E361D3060184E361F3068A0435E688D
:101D100006F4003606B12043134E361F3060361FDE
:101D20003068A0435E6806F4803606B120430E4E4C
:101D3000083E3060491C1029FFF426AFF8BD0000B2
:101D400044380240083801400000024000040240CC
:101D500000080240000C0240001002400014024043
:101D600000180240001C0240083C014010B54269C6
:101D700021EA020302EA010443EA0443836110BD3D
:101D80000AB1816101E00B0483617047014800687A
:101D9000704700003400002070B504460CB90120E3
:101DA00070BD4CF6CC402168086045F25550216862
:101DB0000860D4E9001048602168A0688860FFF7D7
:101DC000E5FF05460BE0FFF7E1FF401B312806D990
:101DD0002068C06800F0030008B10320E0E7206835
:101DE000C06800F003000028EDD14AF6AA2021685F
:101DF00008600020D4E701464AF6AA200A6810606D
:101E000000207047034800680349097808440149E5
:101E100008607047340000203C00002010B50D48D9
:101E2000006840F400700B4908600846006840F400
:101E3000806008600846006840F4807008600320F5
:101E400000F0DCF80F2000F007F800F05FF8002049
:101E500010BD0000003C02402DE9F04188B004466E
:101E60000027B84600BF002001902348006840F0DA
:101E70001000214908600846006800F01000019039
:101E800000BF00BF02A903A800F08EF9069F1FB98A
:101E900000F0B2F9054602E000F0AEF9450017483F
:101EA000B5FBF0F0A0F1010815481649086040F2B2
:101EB000E7311448C160C0F80480002101618160ED
:101EC000816100F0BBFC064696B90E4800F01CFD8F
:101ED00006466EB9362000F043F8102C07D20022D7
:101EE0002146362000F04CF80748046000E0012647
:101EF000304608B0BDE8F0814038024040420F0053
:101F0000001000401C0900203800002008B500BF68
:101F1000002000901148006840F480400F4908609C
:101F20000846006800F48040009000BF00BF00BF7A
:101F300000200090081F006840F08050091F0860D2
:101F40000846006800F08050009000BF00BF0022EB
:101F50000F21901E00F014F808BD00004438024024
:101F600001460846002809DB00F01F0301229A40C1
:101F700043099B0003F1E023C3F8002100BF704731
:101F80002DE9F05F80460D461646002703F076FDEA
:101F9000074639462A46334601F00700C0F1070AD2
:101FA000BAF1040F02D94FF0040A01E0C0F1070AA8
:101FB000D14600F1040ABAF1070F02D24FF0000A2D
:101FC00001E0A0F1030AD4464FF0010A0AFA09FA27
:101FD000AAF1010A0AEA020A0AFA0CFA4FF0010B06
:101FE0000BFA0CFBABF1010B0BEA030B4AEA0B04F7
:101FF0002146404603F04AFDBDE8F09F00BF00F0D7
:102000000702064B19684FF6FF031940044B0B43B8
:1020100043EA0221014B196000BF70470CED00E05C
:102020000000FA0570B504460D460CB9012070BDDC
:102030005848006800F00700A84209D255490D70C1
:102040000846006800F00700A84201D00120EEE732
:10205000207800F0020002281DD1207800F0040052
:10206000042805D14C48006840F4E0504A49086013
:10207000207800F00800082805D14748006840F49F
:102080006040454908604448006820F0F000A168BD
:10209000084341490860207800F00100A8B3606857
:1020A000012807D13C4808380068C0F34040B8B95F
:1020B0000120BCE76068022802D06068032807D1CD
:1020C000354808380068C0F3406048B90120AEE7E1
:1020D000314808380068C0F3400008B90120A6E77D
:1020E0002D48006820F00300616808432A49086011
:1020F000FFF74CFE064609E0FFF748FE801B41F261
:102100008831884202D9032091E707E0224800681D
:1021100000F00C006168B0EB810FEDD11D48006844
:1021200000F00700A84209D91A490D700846006856
:1021300000F00700A84201D0012078E7207800F0E5
:102140000400042807D11448006820F4E050E16836
:10215000084311490860207800F00800082808D1D9
:102160000D48006820F46040216940EAC1000A4936
:10217000086000F061F808490968C1F30311074AD3
:10218000515CC8400649086006480068FFF764FED5
:1021900000204CE7003C024008380240C4800008A0
:1021A00040000020380000200F2202600D4A126813
:1021B00002F0030242600B4A126802F0F0028260F1
:1021C000084A126802F4E052C260064A126802F439
:1021D0006042D2080261044A126802F007020A60F3
:1021E0007047000008380240003C02400148006887
:1021F000704700004000002000B5FFF7F7FF0449DA
:102200000968C1F38221034A515CC84000BD000047
:1022100008380240D480000800B5FFF7E7FF044902
:102220000968C1F34231034A515CC84000BD000057
:1022300008380240D48000082DE9F047002400252A
:102240000026A1462548006800F00C0020B10428B3
:1022500005D008283AD105E0DFF8849039E0DFF8AE
:10226000849036E01D48001F006800F03F041B48C2
:10227000001F006800F4800078B11A481749091F50
:102280000968C1F38811A0FB0170014622460023B2
:102290003846FDF7F5FF05460EE011480F49091FC6
:1022A0000968C1F38811A0FB017001462246002392
:1022B0003846FDF7E5FF05460848001F0068C0F3F3
:1022C0000140401C4600B5FBF6F902E0DFF8109033
:1022D00000BF00BF4846BDE8F08700000838024054
:1022E0000024F40000127A00F8B504460CB901206D
:1022F000F8BD207800F00100002874D0F94800688B
:1023000000F00C0004280DD0F648006800F00C0026
:10231000082813D1F348001F006800F48000B0F5CE
:10232000800F0BD1EF4808380068C0F34040002808
:1023300059D06068002856D10120D9E700BF6068F5
:10234000B0F5803F08D1E7480838006840F4803095
:10235000E449083908601EE06068B0F5A02F0DD18F
:10236000E0480838006840F48020DE4908390860F9
:102370000846006840F4803008600CE0D94808380E
:10238000006820F48030D7490839086008460068A2
:1023900020F48020086000BF606890B1FFF7F6FC71
:1023A000054606E0FFF7F2FC401B642801D9032034
:1023B0009EE7CC4808380068C0F340400028F1D0C0
:1023C00011E0FFF7E3FC054606E0FFF7DFFC401BEA
:1023D000642801D903208BE7C24808380068C0F39D
:1023E00040400028F1D1207800F0020002285FD19F
:1023F000BC48006800F00C0058B1BA48006800F012
:102400000C0008281CD1B748001F006800F48000A9
:10241000B0B9B44808380068C0F3400020B1E068A3
:10242000012801D0012063E7AE480838006820F099
:10243000F800216940EAC100AA490839086037E07C
:10244000E06800B30120A8490860FFF79FFC05463B
:1024500006E0FFF79BFC401B022801D9032047E759
:10246000A04808380068C0F340000028F1D09D481B
:102470000838006820F0F800216940EAC100994955
:102480000839086014E0002097490860FFF77EFCD7
:10249000054606E0FFF77AFC401B022801D903201D
:1024A00026E7904808380068C0F340000028F1D1C2
:1024B000207800F0080008282CD16069A8B101201C
:1024C0008A490860FFF762FC054606E0FFF75EFCFC
:1024D000401B022801D903200AE782486C300068BB
:1024E000C0F340000028F1D014E000207F490860CC
:1024F000FFF74CFC054606E0FFF748FC401B0228AE
:1025000001D90320F4E677486C300068C0F340003E
:102510000028F1D1207800F00400042870D10027B1
:1025200070483830006800F0805090B900BF00203B
:1025300000906C483830006840F08050694938316C
:1025400008600846006800F08050009000BF00BF9F
:1025500001276748006800F48070B0B964480068DB
:1025600040F4807062490860FFF710FC054606E001
:10257000FFF70CFC401B022801D90320B8E65C4899
:10258000006800F480700028F2D000BFA068012825
:1025900008D154486830006840F001005149683162
:1025A00008601DE0A06805280DD14E48683000681D
:1025B00040F004004B49683108600846006840F06C
:1025C000010008600CE047486830006820F0010016
:1025D0004449683108600846006820F0040008603B
:1025E00000BFA068A8B1FFF7D1FB054609E0FFF7DF
:1025F000CDFB401B41F28831884202D9032077E6A7
:1026000026E0384868300068C0F340000028EED06B
:1026100013E0FFF7BBFB054608E0FFF7B7FB401BE5
:1026200041F28831884201D9032061E62D486830A3
:102630000068C0F340000028EFD1012F07D12948DE
:102640003830006820F0805026493831086000BFDB
:10265000A069002845D02348006800F00C00082835
:102660005DD0A069022845D100201F490866FFF708
:102670008DFB054606E0FFF789FB401B022801D9C8
:10268000032035E6174808380068C0F3406000288A
:10269000F1D1D4E907010843616A40EA81110122BE
:1026A000A06AC2EB500041EA00412C20005D41EAE3
:1026B00000600C49091F086001200B490866FFF7FC
:1026C00065FB054606E0FFF761FB401B022801D9C8
:1026D00003200DE6034808380068C0F34060002876
:1026E000F1D049E00838024000004742800E4742DE
:1026F00000700040002021490866FFF747FB0546AF
:1027000006E0FFF743FB401B022801D90320EFE559
:102710001B480068C0F340600028F2D12CE0A0699B
:10272000012800D1E4E51648001D0668A0690128CB
:1027300020D006F48001E06981421BD106F03F0100
:10274000206A814216D147F6C0703040616AB0EB12
:10275000811F0FD106F440310122A06AC2EB500064
:10276000B1EB004F06D106F070612C20005DB1EB9B
:10277000006F01D00120BBE50020B9E50000474211
:10278000003802407047704730B502460B4600BF24
:1027900092F83C00012801D1022030BD012082F8CE
:1027A0003C0000BF022082F83D00106844681068B9
:1027B000816824F070041868044310684460184D60
:1027C0001068A8421BD01068B0F1804F17D0154D8B
:1027D0001068A84213D0144D1068A8420FD0134DB2
:1027E0001068A8420BD0124D1068A84207D0114DB6
:1027F0001068A84203D0104D1068A84205D121F0FE
:1028000080015868014310688160012082F83D0012
:1028100000BF002082F83C0000BF00BFBDE7000001
:10282000000001400004004000080040000C00408F
:1028300000040140004001400018004010B504466B
:102840000CB9012010BD94F83D0028B9002084F88F
:102850003C00204600F026F8022084F83D00211DAF
:10286000206802F02DF9012084F8460000BF84F8AA
:102870003E0001213F2001554020015541200155D6
:1028800000BF00BF012084F84200432001554420CE
:1028900001554520015500BF012084F83D0000206E
:1028A000D0E7000008B5154A016891420FD100BF7A
:1028B000002100911249096841F00401104A116099
:1028C0001146096801F00401009100BF15E00D4AAE
:1028D0000168914211D100BF002100910849091DF2
:1028E000096841F48031064A121D116011460968D9
:1028F00001F48031009100BF00BF08BD0008004016
:102900004038024000400140014691F83D00012856
:1029100001D001207047022081F83D000868C0689E
:1029200040F001000B68D8601A4B086898421BD031
:102930000868B0F1804F17D0174B0868984213D041
:10294000164B086898420FD0154B086898420BD078
:10295000144B0868984207D0134B0868984203D07C
:10296000124B086898420CD10868806800F0070292
:10297000062A0CD00868006840F001000B68186057
:1029800005E00868006840F001000B68186000204E
:10299000C0E70000000001400004004000080040C3
:1029A000000C0040000401400040014000180040BD
:1029B0002DE9F04104460D46002700BF94F83C0085
:1029C000012802D10220BDE8F081012084F83C00FA
:1029D00000BF022084F83D002068866826F0770654
:1029E00026F47F46206886602868502833D00CDCA7
:1029F000202850D004DC00284BD0102851D149E0C9
:102A0000302849D040284CD139E060282DD070289A
:102A100007D0B0F5805F03D0B0F5005F41D10DE085
:102A200041E0D5E902136A68206802F0C6F8206820
:102A3000866846F077062068866034E0D5E90213A0
:102A40006A68206802F0B9F82068806840F4804025
:102A50002168886027E0EA686968206802F09EF9CA
:102A60005021206802F0B4F81DE0EA686968206827
:102A700002F0A7F96021206802F0AAF813E0EA68E2
:102A80006968206802F08AF94021206802F0A0F805
:102A900009E000BF00BF00BF2968206802F098F875
:102AA00001E0012700BF00BF012084F83D0000BF06
:102AB000002084F83C0000BF384684E7704710B51A
:102AC000044620680069C0F34000D8B12068C0689F
:102AD000C0F34000B0B16FF002002168086101202E
:102AE00020772068806900F0030018B12046FFF7C6
:102AF000E5FF05E0204600F005F9204600F0B9F9B1
:102B00000020207720680069C0F38000D8B12068D9
:102B1000C068C0F38000B0B16FF0040021680861A4
:102B2000022020772068806900F4407018B12046A8
:102B3000FFF7C4FF05E0204600F0E4F8204600F06F
:102B400098F90020207720680069C0F3C000D8B150
:102B50002068C068C0F3C000B0B16FF00800216801
:102B60000861042020772068C06900F0030018B1D4
:102B70002046FFF7A3FF05E0204600F0C3F82046FB
:102B800000F077F90020207720680069C0F300107A
:102B9000D8B12068C068C0F30010B0B16FF0100069
:102BA00021680861082020772068C06900F440701F
:102BB00018B12046FFF782FF05E0204600F0A2F89A
:102BC000204600F056F9002020772068006900F0C8
:102BD000010058B12068C06800F0010030B16FF00A
:102BE000010021680861204600F0CAF920680069E8
:102BF000C0F3C01058B12068C068C0F3C01030B135
:102C00006FF08000216808612046FFF7BBFD206857
:102C10000069C0F3801058B12068C068C0F380100C
:102C200030B16FF0400021680861204600F0CAF919
:102C300020680069C0F3401058B12068C068C0F334
:102C4000401030B16FF02000216808612046FFF786
:102C50009AFD10BD10B586B00446142101A8FDF7F9
:102C600059FB2349206888421ED100BF00200090F4
:102C70002048006840F008001E49086008460068C7
:102C800000F00800009000BF00BF4FF440400190EA
:102C9000022002900020039004900220059001A9D8
:102CA0001548FEF769FF20E01449206888421CD1CE
:102CB00000BF002000900F48006840F010000D4950
:102CC00008600846006800F01000009000BF00BFD8
:102CD00060200190022002900020039004900320C5
:102CE000059001A90648FEF747FF06B010BD000099
:102CF0000008004030380240000C02400040014013
:102D00000010024070472DE9F04104460D4616467A
:102D1000002700BF94F83C00012802D10220BDE842
:102D2000F081012084F83C0000BF36B1042E1BD096
:102D3000082E31D00C2E5ED145E02946206801F0E6
:102D400051FF2068806940F0080021688861206890
:102D5000806920F004002168886120688069296901
:102D600008432168886148E02946206801F072FF25
:102D70002068806940F4006021688861206880696B
:102D800020F480602168886120688069296940EAB0
:102D900001202168886130E02946206801F098FF11
:102DA0002068C06940F008002168C8612068C069D7
:102DB00020F004002168C8612068C06929690843BF
:102DC0002168C86119E02946206801F0BDFF20682C
:102DD000C06940F400602168C8612068C06920F4BF
:102DE00080602168C8612068C069296940EA0120C3
:102DF0002168C86101E0012700BF00BF00BF0020BB
:102E000084F83C0000BF384689E710B504460CB989
:102E1000012010BD94F83D0028B9002084F83C0042
:102E2000204600F025F8022084F83D00211D20688E
:102E300001F046FE012084F8460000BF84F83E0001
:102E400001213F200155402001554120015500BF7F
:102E500000BF012084F84200432001554420015561
:102E60004520015500BF012084F83D000020D0E737
:102E70007047704770B504460D4615B994F83E008A
:102E80000BE0042D02D13F20005D06E0082D02D1A9
:102E90004020005D01E04120005D012801D00120BB
:102EA00070BD1DB9022084F83E000EE0042D03D150
:102EB00002213F20015508E0082D03D102214020C6
:102EC000015502E0022141200155012229462068D6
:102ED00001F062FE23492068884203D0224920681D
:102EE000884201D1012000E0002028B12068406C18
:102EF00040F40040216848641A49206888421BD089
:102F00002068B0F1804F17D018492068884213D04C
:102F10001749206888420FD01649206888420BD094
:102F200011492068884207D013492068884203D09D
:102F30001249206888420CD12068806800F007069A
:102F4000062E0CD02068006840F00100216808605F
:102F500005E02068006840F001002168086000205A
:102F60009EE7000000000140000401400004004012
:102F700000080040000C00400040014000180040E4
:102F800010B5044603492068884201D1FEF73AFF94
:102F900010BD00000010004010B500210748FFF7E9
:102FA00069FF04210548FFF765FF08210448FFF782
:102FB00061FF0C210248FFF75DFF10BD800100207A
:102FC000380100207047704770B50446002520681E
:102FD0004069C0F3C01594F83D00212817D1B5B160
:102FE00000BF00BF2168143151E8001F21F08000AC
:102FF0002168143141E80002002AF3D100BF606B60
:1030000010B1606BFEF759FB204602F058F82068BB
:103010004069C0F3801594F83E00222817D1B5B15D
:1030200000BF00BF2168143151E8001F21F04000AB
:103030002168143141E80002002AF3D100BFA06BDF
:1030400010B1A06BFEF739FB204601F0F2FF002023
:1030500070BD70472DE9F84F044620680568206868
:10306000C668206847694FF00009CA4605F00F0995
:10307000B9F1000F0AD105F0200038B106F02000A8
:1030800020B1204602F02EF8BDE8F88FB9F1000F0C
:103090007CD007F0010018B906F49070002875D0B4
:1030A00005F0010030B106F4807018B1206C40F0DA
:1030B0000100206405F0040030B107F0010018B1F0
:1030C000206C40F00200206405F0020030B107F0EF
:1030D000010018B1206C40F00400206405F00800E5
:1030E00048B106F0200010B907F0010018B1206CBB
:1030F00040F008002064206C002846D005F0200035
:1031000028B106F0200010B1204601F0EBFF206846
:103110004069C0F3801A206C00F0080010B9BAF1C1
:10312000000F2DD0204601F084FF2068406900F098
:103130004000402820D100BF00BF2168143151E871
:10314000001F21F040002168143141E80002002AEC
:10315000F3D100BFA06B50B17548A16B0865A06B9F
:10316000FEF701FB88B1A06B016D88470DE020469A
:10317000FFF76FFF09E009E02046FFF76AFF04E070
:103180002046FFF766FF002020647DE7206B0128C2
:1031900076D105F01000002872D006F0100000284B
:1031A000FAD000BF002000902068006800902068DE
:1031B0004068009000BF00BF2068406900F04000F8
:1031C00040285ED1A06B006840681FFA80F8B8F113
:1031D000000F54D0A08D404551DDA4F82E80A06B87
:1031E000C069B0F5807F43D000BF00BF21680C31BB
:1031F00051E8001F21F4807021680C3141E8000281
:10320000002AF3D100BF00BF00BF2168143151E88C
:10321000001F21F001002168143141E80002002A5A
:10322000F3D100BF00BF00BF2168143151E8001F77
:1032300021F040002168143141E80002002AF3D156
:1032400000BF202084F83E000020206300BF00BFA4
:1032500021680C3151E8001F21F0100021680C3169
:1032600041E80002002AF3D100BFA06BFEF725FA67
:10327000A08DE28D801A81B22046FFF7A4FE03E7FD
:1032800040E0A08DE18D401A1FFA80F8E08DC0B3B8
:10329000B8F1000F35D000BF00BF21680C3151E8F4
:1032A000001F21F4907021680C3141E80002002ACF
:1032B000F3D100BF00BF00BF2168143151E8001FE7
:1032C00021F001002168143141E80002002AF3D105
:1032D00000BF202084F83E000020206300BF00BF14
:1032E00021680C3151E8001F21F0100021680C31D9
:1032F00041E80002002AF3D100BF41462046FFF713
:1033000062FEC1E605F0800030B106F0800018B121
:10331000204602F0E1F8B7E605F0400030B106F0D3
:10332000400018B1204601F0BAFEADE600BFABE6A2
:10333000FF4E000810B504460CB9012010BDA0696D
:1033400000B100E000BF94F83D0028B9002084F8E7
:103350003C00204600F028F8242084F83D00206836
:10336000C06820F400502168C860204601F036FF94
:103370002068006920F49040216808612068406955
:1033800020F02A00216848612068C06840F400509D
:103390002168C86000202064202084F83D0084F863
:1033A0003E000020CAE7000010B586B00446142194
:1033B00001A8FCF7AFFF5F492068884259D100BFE0
:1033C000002000905C48006840F010005A490860F6
:1033D0000846006800F01000009000BF00BF00BF6A
:1033E0000020009054481438006840F00100524911
:1033F000143908600846006800F00100009000BF22
:1034000000BF4FF4C06001900220029000200390A2
:10341000032004900720059001A94848FEF7ACFB63
:103420004748484908604FF000604860002145481F
:103430008160C1604FF4806101610021416181615F
:103440004FF48071C161002101624162FEF7C0FA50
:1034500008B1FDF7C3FB00BF3A48A063846300BF17
:10346000002205212520FEF78BFD2520FEF778FDA3
:103470005EE03549206888425AD100BF00200090A4
:103480002D48001F006840F480202B49091F086068
:103490000846006800F48020009000BF00BF00BF15
:1034A0000020009024481438006840F002002249AF
:1034B000143908600846006800F00200009000BF60
:1034C00000BF4FF440600190022002900020039062
:1034D000032004900720059001A91C48FEF74CFB2F
:1034E0001B481C4908604FF00060486000211948E3
:1034F0008160C1604FF4806101610021416181619F
:103500004FF48071C161002101624162FEF760FAEF
:1035100008B1FDF763FB00BF0E48A063846300BFE2
:10352000002205212720FEF72BFD2720FEF718FD9E
:1035300006B010BD001001404438024000000240B7
:10354000406402405C080020004800400004024043
:1035500028600240BC08002070B504460D4616469F
:1035600094F83E00202816D105B10EB9012070BD97
:1035700000BF94F83C00012801D10220F7E70120A8
:1035800084F83C0000BF00202063324629462046D4
:1035900001F03AFFEBE70220E9E770477047704718
:1035A00000BFFEE770B504460D46012C08D10C2083
:1035B00047490860C00348604FF4A00088601CE0E1
:1035C000022C07D10C204249086080034860E004C7
:1035D000886012E0032C08D103203D4908604FF4B5
:1035E000002048602005886007E00C20384908600A
:1035F000C00348604FF4A000886036483649086030
:10360000334800684860002133488160C160304819
:103610004168314801612E4881682F48416100218D
:10362000017641768176C17601774177FDF740FEDC
:1036300008B1FDF7D3FA012D09D10C202449C86047
:10364000C103234801614FF4A00141611FE0022D35
:1036500008D10C201E49C86081031D480161E9049E
:10366000416114E0032D09D103201949C8604FF4CA
:103670000021174801612905416108E00C20144927
:10368000C860C103124801614FF4A00141611348B1
:10369000134908600E48C0684860002110488160E6
:1036A000C1600B4801690E480161094841690C4835
:1036B00041610021017641768176C17601774177BB
:1036C000FDF7F6FD08B1FDF789FAFDF753F870BD77
:1036D0001401002000640040C40000200068004085
:1036E000EC00002008B500BF0020009016480068DC
:1036F00040F48000144908600846006800F4800027
:10370000009000BF00BF00BF002000900846006886
:1037100040F4001008600846006800F400100090B3
:1037200000BF00BF002205210C20FEF729FC0C2061
:10373000FEF716FC002205213A20FEF721FC3A2074
:10374000FEF70EFC08BD00003038024010B50F4BEC
:10375000002201210E4802F007FB0E4908600E4AC4
:1037600000210E4802F0A2FA0D4908600D4A00211E
:103770000D4802F09BFA0D4908600D4A00210D48E2
:1037800002F094FA0C49086010BD0000AC800008FB
:10379000F507000810000020408000089949000843
:1037A0000400002064800008EB4D000808000020A1
:1037B00088800008154E00080C00002000B587B076
:1037C000142102A8FCF7A6FD00BF002001903E488E
:1037D000006840F010003C4908600846006800F0AE
:1037E0001000019000BF00BF00BF002001900846FC
:1037F000006840F0800008600846006800F0800023
:10380000019000BF00BF00BF002001900846006883
:1038100040F0020008600846006800F002000190D5
:1038200000BF00BF00BF002001900846006840F0C4
:10383000080008600846006800F00800019000BF1A
:1038400000BF00BF002001900846006840F0400023
:1038500008600846006800F04000019000BF00BF0B
:1038600000BF002001900846006840F00100086099
:103870000846006800F00100019000BF00BF01226F
:1038800018211248FEF77CFA00224FF420711048EC
:10389000FEF776FA18200290012003900020049091
:1038A000059002A90948FEF767F94FF420700290CD
:1038B0000120039000200490059002A90448FEF71F
:1038C0005BF907B000BD0000303802400010024034
:1038D0000018024010B507480749086001204860F9
:1038E00040F6FF7104488160FEF756FA08B1FDF713
:1038F00075F910BD003000402C01002000B58DB0DE
:10390000002009900A900B900C90079008901C21C1
:103910006846FCF7FFFC23482349086029204860DB
:103920000021214881606321C16000210161816122
:10393000FEF784FF08B1FDF751F94FF4805009906C
:1039400009A91948FFF734F808B1FDF747F91648F7
:10395000FFF75BFA08B1FDF741F9002007900890E6
:1039600007A91148FEF710FF08B1FDF737F96020ED
:1039700000900020019002900490082269460A48B5
:10398000FFF7C1F908B1FDF729F90C22694606488D
:10399000FFF7B9F908B1FDF721F90348FFF75AF924
:1039A0000DB000BD000800403801002000B58BB00C
:1039B00000200790089009900A901C216846FCF7A7
:1039C000A9FC1E481E4908605320486000211C487D
:1039D00081606321C160002101618161FEF72EFFDA
:1039E00008B1FDF7FBF84FF48050079007A9144881
:1039F000FEF7DEFF08B1FDF7F1F81148FFF705FA11
:103A000008B1FDF7EBF860200090002001900290D3
:103A10000490002269460A48FFF775F908B1FDF7DE
:103A2000DDF8042269460648FFF76DF908B1FDF795
:103A3000D5F80348FFF70EF90BB000BD0040014078
:103A40008001002010B513481349086013484860EE
:103A50004FF48051104881604900C160C910016174
:103A60000C21416100218161C161FFF763FC08B154
:103A7000FDF7B4F808480068C06840F01000064937
:103A80000968C8604FF4007205490348FFF764FDF8
:103A900010BD000000100140D4070020A0860100E6
:103AA000CB01002010B51248124908604FF4E130F4
:103AB000486000210F488160C16001610C214161B3
:103AC00000218161C161FFF735FC08B1FDF786F87F
:103AD00008480068C06840F0100006490968C860DE
:103AE0004FF4007204490348FFF736FD10BD000093
:103AF0000048004018080020D305002000BFFEE762
:103B000000BFFEE710B55148007800F00100B0B9E1
:103B10004F48007890B100231A4603214D4801F028
:103B200097F900231A4604214A4801F091F9002030
:103B300049490870464908704849086010BD444822
:103B4000007898B900231A460321424801F080F911
:103B50002323002204213F4801F07AF901203C4947
:103B6000087003F0D3FF3D490860E7E73848007864
:103B700001280CD103F0CAFF38490968401A40F601
:103B8000B831884200D2D9E7022031490870304864
:103B90000078022858D12D480078C0F34000C0B901
:103BA0002A480078C0F3800098B92B480078012893
:103BB0000FD0322300220321264801F049F91C23AB
:103BC00000220421234801F043F901202249087012
:103BD0003AE01E480078C0F34000C0B11B480078AE
:103BE000C0F3800098B91C48007802280FD0372312
:103BF00000220321174801F02BF938230022042169
:103C0000144801F025F90220134908701CE00F4800
:103C10000078C0F34000B8B90C480078C0F38000C9
:103C200090B10D48007803280ED03C2300220321D8
:103C3000084801F00DF9542300220421054801F041
:103C400007F903200449087000BF77E7240000202B
:103C50001F000020380100201E000020200000204E
:103C600010B51D48807801282CD100201A49887091
:103C700008460088192806DA4FF400711648C01C5F
:103C8000FCF748FB15E000200FE01349C91C0A5C53
:103C900012490B88091DCA54091F0988491CC1F320
:103CA00008010E4A1180411C88B20B4909888142E3
:103CB000EBDC4FF400710848C01CFCF72BFB002024
:103CC000054908804FF400720349C91C0448FFF7F6
:103CD00043FC02F0E3FE10BDC8010020640900208F
:103CE000D40700207E480089F02806D17D4800785E
:103CF00020F001007B49087013E07948008940F208
:103D00000F71884207D17748007820F00100401CED
:103D10007449087005E07348007820F0010071498B
:103D200008706F484089F0280BD16E48007820F069
:103D300002006C4908700846007820F00400087002
:103D40002FE067484089B0F5806F0CD16548007856
:103D500020F00200801C634908700846007820F0BB
:103D6000040008701DE05E48408940F20F718842EF
:103D70000CD15C48007820F002005A4908700846CF
:103D8000007820F00400001D08700AE05548007813
:103D900020F00200534908700846007820F0040023
:103DA00008704F488089F0280BD14E48007820F0E9
:103DB00008004C4908700846007820F01000087090
:103DC0002FE047488089B0F5806F0CD145480078D6
:103DD00020F008000830434908700846007820F0B9
:103DE000100008701DE03E48808940F20F71884243
:103DF0000CD13C48007820F008003A490870084689
:103E0000007820F01000103008700AE03548007883
:103E100020F00800334908700846007820F01000B0
:103E200008702F48C089F02806D12E48007820F06D
:103E300020002C49087013E02948C08940F20F7116
:103E4000884207D12748007820F0200020302549FB
:103E5000087005E02348007820F020002149087010
:103E60001F48008AF02806D11E48007820F0400044
:103E70001C49087013E01A48008A40F20F7188420A
:103E800007D11848007820F04000403015490870EC
:103E900005E01448007820F04000124908701048EE
:103EA000408AF02806D10F48007820F080000D49A4
:103EB000087013E00A48408A40F20F71884207D127
:103EC0000848007820F0800080300649087005E03E
:103ED0000448007820F08000024908707047000014
:103EE000BA0F00202400002010B501F083FB10BDA4
:103EF0002DE9F04104460D46164600BF0E4F3878B6
:103F0000532801D001F076FB00BFEFF31180074684
:103F1000202080F3118800BF00BF3246294620468A
:103F200000F00CF88046F8B280F3118800BF00BFA3
:103F30004046BDE8F0810000B0EA00202DE9F047DE
:103F4000074688461646C24607EB47011B4800EB6A
:103F5000C109D9F8140020B1012811D0022826D1B6
:103F60001EE0484601F07EFB0546B54201D2002422
:103F700005E0344632465146484601F052FD18E00D
:103F8000484601F06FFB0546B54201D2284600E0E5
:103F90003046044622465146484601F042FD08E0BC
:103FA00032465146484601F001FD044601E0002436
:103FB00000BF00BF2046BDE8F0870000C8EA00202F
:103FC0000FB438B5044606A800906A462046059905
:103FD00000F008F8054600200090284638BC5DF83F
:103FE00014FB00002DE9F74F2DED028B98B00D4624
:103FF000144603A8139040201490002015901A989E
:1040000017900020169000BF2E786D1C06B90DE1A8
:10401000252E79D100274FF0010A00BF2E78232EDC
:1040200012D02B2E0CD02D2E02D0302E10D103E02A
:1040300047F001076D1C0EE047F002076D1C0AE017
:1040400047F004076D1C06E047F008076D1C02E00E
:104050004FF0000A00BF00BFBAF1000FDED14FF0F1
:10406000000900BF2E78302E01DB392E00DD07E07D
:104070006D1CA6F1300009EB890100EB4109F1E765
:1040800000BF4FF000082E782E2E10D16D1C00BFFF
:104090002E78302E01DB392E00DD07E06D1CA6F1F5
:1040A000300008EB880100EB4108F1E700BF2E78F3
:1040B00000BF6C2E01D0682E02D16D1C2E7800E05E
:1040C00000E0F6E700BF662E73D008DC252E71D025
:1040D000582E41D0632E0BD0642E6CD115E0702E7B
:1040E0006BD0732E4BD0752E22D0782EF5D132E0C6
:1040F0002168081D2060D1F800A00AF0FF0B594686
:1041000013A801F031FC86E088E02168081D2060DA
:10411000D1F800A0B8F1000F01D027F00207434604
:104120000A22514613A8CDE9009701F031FB72E055
:104130002168081D2060D1F800A0B8F1000F01D05F
:1041400027F0020743460A22514613A8CDE90097FB
:1041500001F094FB5FE000BF2168081D2060D1F8EA
:1041600000A0B8F1000F01D027F00207434610224B
:10417000514613A8CDE9009701F080FB4BE0216880
:10418000081D2060D1F800B0BBF1000F01D10FF283
:10419000C80B00BF9BF800600BF1010B06B906E0ED
:1041A000314613A801F0E0FB16980028F2DA00BFB0
:1041B00031E017E011E02DE0FFE72168081D2060E5
:1041C000D1F800A0002008210B461022CDE90010F4
:1041D000514613A801F052FB1DE0252113A801F060
:1041E000C3FB18E02068C01D20F00700014608301E
:1041F000206091ED000BB0EE408AF0EE608A3B4605
:104200004A464146B0EE480AF0EE680A13A801F0AB
:1042100037FA00E000BF00BF6D1C03E0314613A871
:1042200001F0A2FB16980028BFF6EEAE00BF16986C
:1042300000280ADD159820B103A9159A1A98FFF7EE
:1042400057FEDDE9151008441690169818B0BDEC1D
:10425000028BBDE8FE8F0000284E554C4C29000013
:1042600010B54548408AF0282FD14348008AF028ED
:104270002BD14148C089F02827D13F488089F028B8
:1042800023D13D484089F0281FD13B480089F028C0
:104290001BD13A480078C0B93748408840F2953180
:1042A000884212DD3448408840F25D4188420CDA91
:1042B00031480088B0F5677F07DD2F480088C91DA9
:1042C000884202DA01202D4908702C480078002825
:1042D00051D0FFF707FD2A480078C0F340100028AE
:1042E00047D027480078C0F3C00048B92448007878
:1042F000C0F3001020B94FF4FA702249088021E081
:104300001F480078C0F3C00048B11D480078C0F3D2
:10431000001020B940F2EE201A49088012E0184837
:104320000078C0F3C00048B915480078C0F3001009
:1043300020B14FF47A701349088003E04FF4FA700B
:104340001049088000F028F80F48B0F900300F48F5
:10435000B0F900200E48B0F900100E48B0F9000086
:10436000FCF768FAFFF7CEFB22210348FBF7D2FFE8
:1043700001E0FCF733FB10BDBA0F00202500002040
:104380002400002030000020280000202C00002005
:10439000260000202A0000202DE9F0412DED048B9D
:1043A00084B0002001900290039000250026002791
:1043B00080460024FE48408806B2FD48008805B2C9
:1043C000B5F5677F03DB40F26440854200DD0DB93F
:1043D0004FF0010840F29530864203DB40F25D4029
:1043E000864200DD06B901277FB1B8F1000F0CD07D
:1043F0000020ADF806000021ADF8081010208DF85F
:104400000E0010218DF80F10A2E200208DF80E0092
:1044100000218DF80F10002F63D1B8F1000F60D08C
:1044200040F25D40864227DD40F20F7086420ADB93
:10443000E048008800B2ADF80600DE48008801B20E
:10444000ADF808105EE2A6F25D40DA4909884843FB
:1044500040F2B22190FBF1F000B2ADF80600A6F2F6
:104460005D40D4490988484340F2B22190FBF1F005
:1044700001B2ADF8081045E2002EE3DDB6F5657F28
:10448000E0DCF02E0EDCCB480088C043401C00B2BC
:10449000ADF80600C7480088C043401C01B2ADF823
:1044A00008102FE240F29530801BC249098848432A
:1044B00040F2A52190FBF1F0C043401C00B2ADF8E2
:1044C000060040F29530801BBA490988484340F203
:1044D000A52190FBF1F0C043401C01B2ADF80810DB
:1044E00010E2002F7AD0B8F1000F77D1002D3ADD1D
:1044F000B5F5677F37DAF02D13DCAE49088800EB9D
:10450000D0714910491C09B2ADF80610A9490888B4
:1045100000EBD0716FEA6101491C0AB2ADF80820C6
:10452000F0E1A449088800EBD0714910C5F5677225
:1045300051434FF42B7291FBF2F1491C09B2ADF8D3
:1045400006109C49088800EBD0714910C5F56772C8
:1045500051434FF42B7291FBF2F1C943491C0AB24B
:10456000ADF80820CEE140F26440854299DD40F28A
:104570000F70854211DB8F49088800EBD0716FEA1C
:10458000610109B2ADF806108A49088800EBD071C4
:1045900049100AB2ADF80820B4E18649088800EB5A
:1045A000D0714910A5F26442514340F2AB2291FB15
:1045B000F2F1C94309B2ADF806107E49088800EB54
:1045C000D0714910A5F26442514340F2AB2291FBF5
:1045D000F2F10AB2ADF8082094E1FFE740F25D4045
:1045E00086425ADD002D58DDB5F5677F55DAA6F213
:1045F0005D40C5F56771884220DB6E4909884843F4
:1046000040F2B22190FBF1F4C5F567706043891F59
:1046100090FBF1F0201A00B2ADF80600C5F5677105
:1046200061434FF42B7291FBF2F0C11700EB9171D3
:10463000A4EBA1010AB2ADF8082063E1C5F56770EB
:104640005C49098848434FF42B7190FBF1F4A6F2C2
:104650005D4262438B1D92FBF3F000EBD07221466A
:1046600004EBD1735B10A3EB6202D243521C12B273
:10467000ADF80620A6F25D42624340F2B22392FBFF
:10468000F3F0C21700EB9272921004EBD17302EBBD
:10469000630213B2ADF8083034E140F25D40864267
:1046A00058DDC01D854255DDA6F25D40A5F264418E
:1046B000884220DB3F490988484340F2B22190FB01
:1046C000F1F4A5F26441614340F2AB2291FBF2F0B8
:1046D000C11700EB9171A4EBA10109B2ADF806106E
:1046E000A5F264406043114690FBF1F0201A01B23C
:1046F000ADF8081006E1A5F264402E490988484348
:1047000040F2AB2190FBF1F4A6F25D426243CB1D77
:1047100092FBF3F0C21700EB92729210214604EB69
:10472000D17302EB630212B2ADF80620A6F25D422D
:10473000624340F2B22392FBF3F000EBD07204EB41
:10474000D1735B10A3EB6202D243521C13B2ADF8DB
:104750000830D7E0002E6DDDB6F5657F6ADC002DF0
:1047600068DDB5F5677F65DA40F29530801BC5F5E9
:10477000677188422DDB40F29530801B0D49098816
:10478000484340F2A52190FBF1F4C5F56770604302
:10479000C91D90FBF1F0201AC043401C00B2ADF8D7
:1047A0000600C5F5677161434FF42B7204E0000009
:1047B000BA0F00203000002091FBF2F0C11700EB8F
:1047C0009171A4EBA101C943491C0AB2ADF80820BC
:1047D00098E0C5F567706949098848434FF42B7123
:1047E00090FBF1F440F29532921B6243CB1F92FB97
:1047F000F3F000EBD072214604EBD1735B10A3EB16
:10480000620212B2ADF8062040F29532921B62436A
:1048100040F2A52392FBF3F0C21700EB92729210C4
:1048200004EBD17302EB6302D243521C13B2ADF816
:10483000083067E0002E65DDB6F5657F62DC40F28A
:10484000644085425EDD40F29530811BA5F26440F4
:10485000814227DB40F29530801B48490988484354
:1048600040F2A52190FBF1F4A5F26441614340F2CE
:10487000AB2291FBF2F0C11700EB9171A4EBA10107
:10488000C943491C09B2ADF80610A5F26440604363
:10489000114690FBF1F0201AC043401C01B2ADF864
:1048A00008102FE0A5F2644034490988484340F2DB
:1048B000AB2190FBF1F440F29532921B62438B1FC7
:1048C00092FBF3F0C21700EB92729210214604EBB8
:1048D000D17302EB6302D243521C12B2ADF8062030
:1048E00040F29532921B624340F2A52392FBF3F013
:1048F00000EBD07204EBD1735B10A3EB620213B236
:10490000ADF80830BDF90600FBF728FE41EC190BA5
:104910009FED1B0B53EC102BFBF7AEFD41EC180B7E
:10492000FBF72DFE00B2ADF80600BDF90800FBF75D
:1049300015FE41EC190B9FED120B53EC102BFBF7FE
:104940009BFD41EC180BFBF71AFE01B2ADF8081005
:10495000BDF806000C490880BDF808000B49088026
:104960009DF80E000A4908809DF80F00094908804B
:1049700004B0BDEC048BBDE8F081000030000020E5
:10498000000000000000F03F26000020280000206A
:104990002A0000202C0000204FF4FA71084800681B
:1049A00001F040FA0AE008210648FDF7DFF9064861
:1049B000FDF721FA4FF4487001F022F9F3E7000007
:1049C00010000020001002402C01002010B54FF014
:1049D000E020006903F08AF8012801D002F0D4FC3D
:1049E00010BD000000B593B0302107A8FBF792FC82
:1049F000142102A8FBF78EFC00BF0020019025487F
:104A0000006840F08050234908600846006800F0C4
:104A10008050019000BF00BF00BF002001901E48E1
:104A2000006840F480401C4908600846006800F4B3
:104A30008040019000BF00BF092007904FF48030F4
:104A4000089001200C9002200D9041050E91042148
:104A50000F91A8211091022111910421129107A810
:104A6000FDF742FC08B1FCF7B9F80F2002900220D4
:104A70000390002004904FF4A05005904FF4805014
:104A80000690052102A8FDF7CDFA08B1FCF7A6F8BB
:104A900013B000BD40380240007000400348006879
:104AA00040F47000014908607047000088ED00E0A4
:104AB00010B50248FEF703F810BD00001C090020E5
:104AC00010B50268294B98420ED0B0F1804F0BD040
:104AD000274B984208D0274B984205D0264B984246
:104AE00002D0264B984203D122F070024B681A4341
:104AF0001E4B984220D0B0F1804F1DD01C4B9842E5
:104B00001AD01C4B984217D01B4B984214D01B4B09
:104B1000984211D01A4B98420ED01A4B98420BD0A3
:104B2000194B984208D0194B984205D0184B98421F
:104B300002D0184B984203D122F44072CB681A433A
:104B400022F080034C6943EA040202608B68C3626E
:104B50000B688362054B984202D0084B984201D102
:104B60000B6903630123436110BD00000000014095
:104B70000004004000080040000C00400004014018
:104B8000004001400044014000480140001800403E
:104B9000001C00400020004030B501F01F0501243A
:104BA00004FA05F3046A9C430462046A01F01F05D9
:104BB00002FA05F52C43046230BD30B50C4681681D
:104BC00021F47F4142EA032525432943816030BD1A
:104BD0000A46816821F0700142F0070319438160A1
:104BE0007047000030B5056A25F001050562026ACC
:104BF0004368846924F0700424F003040D682C4396
:104C000022F002028D682A43104DA84200D103E031
:104C10000F4DA84206D100BF22F00802CD682A43FA
:104C200022F00402094DA84202D0094DA84207D142
:104C300023F4807323F400734D692B438D692B4358
:104C4000436084614D684563026230BD00000140ED
:104C50000004014030B5056A25F010050562026ABE
:104C60004368846924F4E04424F440740D6844EA01
:104C7000052422F020028D6842EA0512124DA84256
:104C800000D103E0114DA84207D100BF22F08002FD
:104C9000CD6842EA051222F040020B4DA84202D034
:104CA0000A4DA84209D123F4806323F400634D69BF
:104CB00043EA85038D6943EA8503436084614D6857
:104CC0008563026230BD0000000001400004014025
:104CD00030B5056A25F480750562026A4368C469C7
:104CE00024F0700424F003040D682C4322F40072B5
:104CF0008D6842EA0522124DA84200D103E0114D11
:104D0000A84207D100BF22F40062CD6842EA052222
:104D100022F480620A4DA84202D00A4DA84209D16D
:104D200023F4805323F400534D6943EA05138D693E
:104D300043EA05134360C4614D68C563026230BD38
:104D4000000001400004014030B5056A25F480559B
:104D50000562036A4468C26922F4E04222F44072A8
:104D60000D6842EA052223F400538D6843EA0533B7
:104D7000084DA84202D0084DA84204D124F4804432
:104D80004D6944EA85144460C2614D68056403625C
:104D900030BD0000000001400004014030B50B466A
:104DA0001446026A056A25F001050562816921F051
:104DB000F00141EA041122F00A021A438161026201
:104DC00030BD30B50B461446056A25F01005056266
:104DD0008169026A21F4704141EA043122F0A002A3
:104DE00042EA03128161026230BD002410E0FEF746
:104DF00037FF002001F058FF0546601C84B24EF6D4
:104E00006020844200DB0024052000F0F9FE00BF92
:104E1000EDE70000002417E010210C48FCF7A6FF86
:104E200000F048F8FFF71CFA002001F03DFF0546AE
:104E3000601C84B24EF66020844200DB00244FF4F4
:104E4000FA7000F0DDFE00BFE6E70000001002404F
:104E500070B504460D460021012D06D0022D06D066
:104E6000032D06D0042D08D105E0002007E0042022
:104E700005E0082003E00C2001E03C2000BF00BF5B
:104E8000632B01D9632103E00BB9002100E019462F
:104E900010B9266871630BE0042802D12668B1635B
:104EA00006E0082802D12668F16301E02668316433
:104EB00070BD00000CB509A103C9CDE90001094886
:104EC0000088401C07490880084600884CF2503191
:104ED000884202DD0020034908800CBD40122100F9
:104EE000000000001C00002070B50546284601F0B7
:104EF000A9FD044614B1D4E90010884770BD70B50F
:104F00000546AC6B0020E085E0842046FEF7A1F862
:104F100070BD70B506460025B46B20684069C0F3CB
:104F2000C01594F83D00212805D125B10020E0846A
:104F3000204600F0C4F820684069C0F3801594F85A
:104F40003E00222805D125B10020E085204600F052
:104F500070F8206C40F0100020642046FEF779F8CD
:104F600070BD70B50546AC6B2868006800F48070B1
:104F7000002842D1E08500BF00BF21680C3151E814
:104F8000001F21F4807021680C3141E80002002AE2
:104F9000F3D100BF00BF00BF2168143151E8001FEA
:104FA00021F001002168143141E80002002AF3D108
:104FB00000BF00BF00BF2168143151E8001F21F07D
:104FC00040002168143141E80002002AF3D100BFFB
:104FD000202084F83E00206B01280ED100BF00BFC6
:104FE00021680C3151E8001F21F0100021680C31BC
:104FF00041E80002002AF3D100BF206B012804D150
:10500000A18D2046FDF7DFFF02E02046FEF7C5FA3E
:1050100070BD70B50546AC6B206B012805D1A08D25
:1050200041082046FDF7CFFF02E02046FEF7B6FA22
:1050300070BD00BF00BF02680C3252E8002F22F49E
:10504000907102680C3242E80013002BF3D100BFCC
:1050500000BF00BF0268143252E8002F22F00101A5
:105060000268143242E80013002BF3D100BF016B39
:1050700001290ED100BF00BF02680C3252E8002F98
:1050800022F0100102680C3242E80013002BF3D129
:1050900000BF202180F83E1000210163704710B549
:1050A00004462068C06820F040002168C8602020C5
:1050B00084F83D002046FEF772FA002010BD00BFC4
:1050C00000BF02680C3252E8002F22F0C0010268D3
:1050D0000C3242E80013002BF3D100BF202180F8EE
:1050E0003D107047F8B5044694F83E00222873D16D
:1050F000A068B0F5805F0CD1206950B90025A66A80
:1051000020684068C0F308003080A06A801CA0625C
:1051100015E0A56A0026A068B0F5805F03D0A068FE
:1051200028B9206918B920684068287004E0206810
:10513000406800F07F002870A06A401CA062E08DEB
:10514000401E80B2E085002844D12068C06820F06D
:1051500020002168C8602068C06820F48070216841
:10516000C8602068406920F0010021684861202063
:1051700084F83E00206B012826D10020206300BF68
:1051800000BF21680C3151E8001F21F01000216898
:105190000C3141E80002002AF3D100BF206800680A
:1051A00000F0100010280AD100BF002000902068F5
:1051B0000068009020684068009000BF00BFA18D8B
:1051C0002046FDF700FF02E02046FEF7E6F900204A
:1051D000F8BD01E00020FBE70220F9E72DE9F84FD8
:1051E00004462068006920F44050E16808432168C3
:1051F00008612169A068084361690843E1690843BF
:1052000000902068C06849F20C6188430099084307
:105210002168C8602068406920F44070A169084393
:105220002168486176492068884203D07549206822
:10523000884203D1FCF7F0FF814602E0FCF7DCFF77
:105240008146E069B0F5004F6CD102206168A0FB97
:10525000015003461920A9FB007001462A46384632
:10526000FBF70EF86421B0FBF1F04FEA001A0220C0
:105270006168A0FB01510B461920A9FB00712A4669
:105280003846FAF7FDFF834602206168A0FB015013
:1052900003461920A9FB00712A463846FAF7F0FFA9
:1052A0006421B0FBF1F000EBC00101EB0010ABEBAF
:1052B0008000322101EBC0006421B0FBF1F000F06E
:1052C000F8000AEB400A02206168A0FB0150034687
:1052D0001920A9FB007001462A463846FAF7D0FF8C
:1052E000834602206168A0FB015003461920A9FBF8
:1052F00000712A463846FAF7C3FF6421B0FBF1F08B
:1053000000EBC00101EB0010ABEB8000322101EBA0
:10531000C0006421B0FBF1F000F0070050442168A8
:1053200088606AE004206168A0FB015003461920F0
:10533000A9FB007001462A463846FAF7A1FF8246CB
:1053400004206168A0FB015003461920A9FB0070EE
:1053500001462A463846FAF793FF6421B0FBF1F084
:1053600000EBC00101EB0010AAEB8000322101EB41
:1053700000106421B0FBF1F000F0F00A0420616835
:10538000A0FB017003461920A9FB00513A462846AC
:10539000FAF776FF6421B0FBF1F00AEB001A042063
:1053A0006168A0FB01510B461920A9FB00712A4638
:1053B0003846FAF765FF834604206168A0FB015078
:1053C00003461920A9FB007001462A463846FAF721
:1053D00057FF6421B0FBF1F000EBC00101EB0010BE
:1053E000ABEB8000322101EB00106421B0FBF1F047
:1053F00000F00F00504421688860BDE8F88F00007D
:10540000001001400014014077B581B004461546F4
:105410000298A062A58500202064222084F83E0026
:105420002A48A16BC8632A48A16B08642948A16B6C
:10543000C8640020A16B086502AE32682368191D9C
:105440002B46A06BFCF73AFB00BF002000902068C1
:105450000068009020684068009000BF00BF00BF57
:10546000002084F83C0000BF206970B100BF00BF7D
:1054700021680C3151E8001F41F4807021680C3123
:1054800041E80002002AF3D100BF00BF00BF21683D
:10549000143151E8001F41F001002168143141E846
:1054A0000002002AF3D100BF00BF00BF2168143101
:1054B00051E8001F41F040002168143141E800022A
:1054C000002AF3D100BF002004B070BD634F000874
:1054D00013500008134F0008014691F83D002128A1
:1054E00028D18868B0F5805F0BD1086948B90A6A8D
:1054F0001088C0F308000B685860086A801C0862B6
:1055000005E00B6A581C086218780B685860C88C54
:10551000401E80B2C88458B90868C06820F0800076
:105520000B68D8600868C06840F040000B68D8601D
:10553000002070470220FCE738B5002511480068BC
:105540000068C0F30015CDB100BF002000900D48E9
:105550000068006800900B4800684068009000BF39
:1055600000BF0848FDF730FD07480068406884B276
:10557000C4F5007005490880012088700148FDF7D6
:1055800069FD38BDD40700205C080020C801002058
:1055900038B50025134800680068C0F30015E5B170
:1055A00000BF002000900F480068006800900D4880
:1055B00000684068009000BF00BF0A48FDF704FD86
:1055C00009480068406884B2C4F500700749A1F832
:1055D00008040121054880F80A140248FDF73AFD45
:1055E00038BD000018080020BC080020C8010020B9
:1055F00000BFFEE770B5144CA8212046FAF78AFEDA
:1056000003202061606111A0A0611349E1614FF4A2
:10561000806121620021A1626162E1620BA02066CB
:105620000E4961661021A16600212167E16661676C
:10563000002505E0C5F10F000949085C60556D1CA7
:10564000102DF7D370BD0000B0EA00205465726DD4
:10565000696E616C0000000058EB002058EF0020DC
:10566000EC80000810B501460A69CB689A4204D85C
:105670008C68641EE41AA01801E0D41A601E10BDE4
:105680002DE9F0472DED068B82B00446B0EE409A2E
:10569000F0EE609A0D4616461F4651EC190BFAF7CC
:1056A0006EFF82465046FAF759FF41EC1A0B53EC55
:1056B000192BFAF7DEFE41EC180B9FED2F0B53EC84
:1056C000102B51EC180BFAF779FF05D251EC180B9F
:1056D00081F0004141EC180B9FED290B53EC102B8E
:1056E00051EC180BFAF721FE41EC180B00230A22AB
:1056F00051462046CDE9006700F04AF8E0680028EE
:1057000003DB2E21204600F02FF9E06800282EDB75
:10571000092D00D909254FF0000825E09FED1A0B4F
:1057200053EC102B51EC180BFAF7A6FE41EC180BBA
:1057300051EC180BFAF723FF814609F13000C1B292
:10574000204600F011F94846FAF708FF41EC1A0B21
:1057500053EC182BFAF78DFE41EC180BE06800288B
:1057600000DA03E008F10108A845D7D300BF02B072
:10577000BDEC068BBDE8F0870000000000000000D3
:10578000BBBDD7D9DF7CDB3D00000000000024401A
:105790002DE9FC5F06460F4692469846DDE90C452A
:1057A000002F01DA784200E0384683464FF00109C5
:1057B00003E09BFBFAFB09F10109D345F9DAC8457F
:1057C00000D9C14634B1002F03DB05F004000428E2
:1057D00000D1641E05F0020010B1B8F1000F11D025
:1057E00005F0010070B96CB108E0641E202130465C
:1057F00000F0BAF8F068002800DA02E00CB1A14528
:10580000F3D300BFF068002836DB002F05DA7F42B3
:105810002D21304600F0A8F807E005F00400042828
:1058200003D12B21304600F09FF8F068002823DBDD
:1058300005F00200022814D105F0010088B9B8F182
:10584000000F0ED16CB108E0641E3021304600F02C
:105850008BF8F068002800DA02E00CB1A145F3D320
:1058600000BFF068002807DB434652463946304601
:10587000CDE9004500F002F8BDE8FC9F2DE9FC5F92
:105880008046894615461E460C9CCDF8049001279B
:10589000BB4605E00198B0FBF5F001900BF1010B60
:1058A0000198A842F6D25E4500D9B3460D9800F0A3
:1058B0000100D0B9CCB10D9800F00200022803D14C
:1058C00016B93020009001E02020009009E0641E0D
:1058D0004046009900F048F8D8F80C00002800DA9B
:1058E00002E00CB1A345F2D300BFD8F80C000028A9
:1058F00035DB09E0012E01D9761E04E0B9FBF7FA89
:10590000AA4500D201E06F43F4E700BF00BFB9FB36
:10591000F7FA0AFB1799134810F80A10404600F0EE
:1059200023F8D8F80C00002800DA03E0B7FBF5F7FD
:10593000002FECD100BF0D9800F0010078B174B1D8
:1059400009E0641E2021404600F00EF8D8F80C0053
:10595000002800DA02E00CB1A345F2D300BFBDE895
:10596000FC9F0000FD80000870B504460E46A56847
:10597000681C6168814206D320684655681CA06097
:10598000E068401CE060D4E9011088420DD1A268B3
:1059900021682069FEF7ACFAA168884203D04FF075
:1059A000FF30E06001E00020A06070BD2DE9F05FF5
:1059B0000446894617464FF0000AE56800BFD4F850
:1059C0001080A84503D9A8EB0500461E04E0A5EB0E
:1059D0000800401CA1680E1AA068401BB04201D903
:1059E000304601E0A068401B0646BE4201D2304668
:1059F00000E038460646606800EB050B3246494633
:105A00005846FAF76EFCB244B144BF1B3544A06857
:105A1000A84200D10025E560002FD0D15046BDE856
:105A2000F09F2DE9F047044689461546E668A068D0
:105A3000871BAF420AD9606800EB060A2A4649462E
:105A40005046FAF74EFC7019E06014E0B846606802
:105A500000EB060A424649465046FAF742FCA5EBDF
:105A60000708D4F804A009EB070142465046FAF7AC
:105A700038FCC4F80C80BDE8F087000002480068DC
:105A8000C0F30220704700000CED00E010B50028C4
:105A900004DB0A07130E054A135406E00A07140E26
:105AA000034A00F00F031B1FD45410BD00E400E0B4
:105AB00018ED00E0EFF30580704702E008C8121F00
:105AC00008C1002AFAD170477047002001E001C1E7
:105AD000121F002AFBD170472DE9F04389B0074619
:105AE0000C4615461E46DDF840804FF0000925485B
:105AF000006800F0806010B10120029013E021489E
:105B0000006800F0006010B1022002900BE01D4818
:105B1000006800F0805010B10420029003E0FF20E4
:105B200009B0BDE8F08300211748029A00EB02108B
:105B300001600CB9894603E0012C01D14FF0040942
:105B400003950495CDF8149000200690CDF81C80A4
:105B500002AB324603A93846FBF758F848B10BA010
:105B60000BA30BA20BA100900020FEF729FA012045
:105B7000D6E700BF3846FBF759FA0328FAD10020D0
:105B8000CEE7000008640040806500401B5B306D7C
:105B900000000000202573257343414E2073656E7D
:105BA0006420746573742064617461206661696C3B
:105BB000210A202573000000FEF796F9FCF72EF964
:105BC000FEF710FFFDF7FAFDFDF78CFDFDF782FEF5
:105BD000FDF7ECFEFDF736FFFDF764FFFDF78EFEE7
:105BE00002210846FDF7DEFCFDF7D6F9FAF79EFD27
:105BF00000F016F8FDF7AAFD00F028F800BFFEE758
:105C000070B50546FFF756FF10B16FF0050404E0CC
:105C1000002415B1284601F0CFF9204670BD0000E0
:105C200010B5FFF747FF10B16FF0050409E0064813
:105C3000006820B9012004490860002401E04FF009
:105C4000FF34204610BD00009400002070B5FFF71F
:105C500031FF10B16FF005041FE011480068012802
:105C600019D100BF801F0021002804DB0A07130E92
:105C70000C4A135406E00A07150E0B4A00F00F03F6
:105C80001B1FD55400BF00BF02200549086001F06A
:105C90000FFA002401E04FF0FF34204670BD0000F1
:105CA0009400002000E400E018ED00E02DE9FF473B
:105CB00080468946144600200390FFF7FBFE00282B
:105CC0004FD1B8F1000F4CD04FF4807618258246A2
:105CD000471E44B3206808B1D4F800A0A06900B101
:105CE000A5692DB1382D03D8207900F0010018B135
:105CF000002004B0BDE8F087606908B160698608DB
:105D0000A06840B1E0685C2805D3206918B16069DB
:105D100008B1012708E0A06830B9E06820B920691F
:105D200010B9002700E00027012F0CD12169A068DD
:105D30004B463246CDE9005102905146404601F0B3
:105D400077FE03900DE067B903A8B2B24B46514607
:105D5000CDE90050404601F039FE012801D0002075
:105D600003900398C5E700002DE9FE4F06468946DB
:105D700092461C4600200290FFF79CFE00284BD163
:105D8000002E49D0082000F0B7FD0546002D43D075
:105D90002E60C5F804A0B9F1000F01D1002700E082
:105DA00001274FF0FF384FF0000B94B1206808B185
:105DB000D4F800B0A06828B1E0682C2802D34FF0D6
:105DC000010808E0A06830B9E06820B94FF0000889
:105DD00001E04FF00008B8F1010F0BD11049A068A5
:105DE0002B463A46CDE900100121584602F071F8E1
:105DF00002900BE0B8F1000F08D109482B463A4653
:105E000001210090584602F049F80290029818B912
:105E100015B1284600F0F2FF0298BDE8FE8F0000A1
:105E2000E94E0008F8B505460E462F46FFF742FE3C
:105E300010B16FF0050411E017B96FF003040DE025
:105E400000200346324604210090384602F0B6F89E
:105E5000012801D1002401E06FF002042046F8BDC2
:105E60002DE9F04105460E461648076816480068B9
:105E7000001D00F005FF681C38B936B112480168F2
:105E8000091D124800F066FF1AE07C190E480068F0
:105E90004460BC4207D20C480168091D0C480068E8
:105EA00000F03EFF0CE008480168091D0948006841
:105EB00000F036FF08480068844201D206480460BA
:105EC000BDE8F0815800002044000020CC140020E0
:105ED0004C000020480000207400002010B504464B
:105EE00000F044FF24480068401C23490860234810
:105EF000006840B9214804600846006801280DD1B7
:105F000000F02AFA0AE01E48006838B91B48006809
:105F1000C06AE16A884201D81848046019480068DC
:105F2000401C184908600846006860641649E06A29
:105F30000968884202D91449E06A0860E16A01EB05
:105F40008101124A02EB8100211D00F003FF00F0E5
:105F500037FF0B48006868B108480068C06AE16A0A
:105F6000884207D24FF0805009490860BFF34F8F35
:105F7000BFF36F8F10BD00005400002044000020CC
:105F800060000020700000205C0000201C10002039
:105F900004ED00E008B500F0E9FE12480068E8B939
:105FA000114800F0ADFE114800F0AAFE0E4810495D
:105FB00008600E480F49086000200F4B0F4A10215F
:105FC00000900A2001F0FAF90649086008460068C6
:105FD00020B10BA10348006800F0B2FF00F0F0FE12
:105FE00008BD000088000020E0140020F414002008
:105FF0008000002084000020081500205815002093
:10600000546D72510000000010B516E000F0AEFEB5
:106010000C48C068C468201D00F032FE0A480068C1
:10602000401E0949086009480068401E0749086089
:1060300000F0C6FE204600F05FF804480068002823
:10604000E4D110BDB81400205400002050000020FE
:1060500070B504460D46206C70B1216CE0680144B7
:10606000E160D4E90210884201D32168E16028464A
:10607000226CE168FAF735F970BD2DE9F04104466C
:106080000F4615464FF00008A66B206C48B92068F3
:1060900000282CD1A06801F0E1FD80460020A0601E
:1060A00025E07DB93946226C6068FAF71AF9216C4F
:1060B000606808446060D4E90101884217D3206811
:1060C000606014E03946226CE068FAF70AF9216C46
:1060D000E068411AE1602168E068884203D2216CDF
:1060E000A068411AE160022D01D106B1761E701C34
:1060F000A0634046BDE8F08110B5044694F859000D
:1061000030B9206B00F07AFE204600F077FE1AE0EE
:1061100094F85900012803D1204600F06FFE12E0E8
:1061200094F85900022801D1012000E0002050B964
:1061300000BF502080F31188BFF34F8FBFF36F8FE4
:1061400000BF00BFFEE710BD0146084A1268126892
:106150000AB9012200E000220A600A6822B9034A53
:106160001268D268106800E00020704780000020AC
:1061700030B54FF44843174800F007042CB1C01D58
:1061800020F00700134C041B1B1B0246124C22601C
:106190000024114D6C60D018083820F007000F4C17
:1061A000206000240D4D2D686C600C4D2D682C6016
:1061B0001146441A4C60094C24680C60084D4C6828
:1061C0002C60084D4C682C604FF00044064D2C604C
:1061D00030BD0000B022002098000020A000002068
:1061E000A8000020A4000020B400002000BFFFF79A
:1061F0000BFF064800680128F9D94FF08050044988
:106200000860BFF34F8FBFF36F8FF0E71C100020C3
:1062100004ED00E02DE9F04106460D46174698468C
:10622000069C0DB9246000E02760E6632564012127
:10623000204601F033F984F84C80BDE8F0812DE967
:10624000F05F82460E4690469B460A9F0C9C4FEAA2
:106250008801A522206BFAF756F8A8F10100216BFE
:1062600001EB800929F0070909F0070008B90120AE
:1062700000E0002050B900BF502080F31188BFF328
:106280004F8FBFF36F8F00BF00BFFEE786B10025C1
:1062900007E0715D04F134004155705D00B902E022
:1062A0006D1C102DF5D300BF00214320015502E0E5
:1062B000002084F83400382F00D33727E762E764E2
:1062C00000202065201D00F028FD04F1180000F0DA
:1062D00024FD2461C7F13800A0616462002060657C
:1062E00084F858005A465146484600F0C1FB2060E9
:1062F0000B9808B10B980460BDE8F09F2DE9F047BA
:1063000006460D4617469846DDE908940DB1012072
:1063100000E0002050B900BF502080F31188BFF387
:106320004F8FBFF36F8F00BF00BFFEE78CB1FFF749
:1063300031FE2660A561C4F81C80C4F82090201DA1
:1063400000F0EBFC2FB194F8280040F0040084F832
:106350002800BDE8F087000010B5002407E004EB3A
:1063600084010F4A02EB810000F0CAFC641C382C47
:10637000F5D30C4800F0C4FC0B4800F0C1FC0B48FE
:1063800000F0BEFC0A4800F0BBFC0A4800F0B8FC74
:1063900004480949086004480849086010BD000025
:1063A0001C1000207C14002090140020A414002055
:1063B000B8140020CC140020480000204C0000201D
:1063C00010B50146164800E0006803688B42FBD315
:1063D0000246436813448B4204D143684C6823440B
:1063E000436001460A464B6813440468A34211D136
:1063F0000C4C03682468A34208D04B6804686468A6
:1064000023444B6003681B680B6005E0054B1B6869
:106410000B6001E003680B60884200D0016010BD92
:1064200098000020A00000202DE9F04104460D4610
:1064300016461F464FF0000865602461B5420CD82F
:10644000F01BA169884202D34FF0010811E0211D21
:106450000948006800F064FC0BE0BE4204D2BD4273
:1064600002D34FF0010804E0211D0448006800F049
:1064700057FC4046BDE8F0818400002080000020E9
:1064800070B5054600F072FCA86B08B9012400E065
:10649000002400F095FC204670BD70B5054600F064
:1064A00065FCA86BE96B884201D1012400E000245F
:1064B00000F086FC204670BDF8B505460F461A4828
:1064C0000068C068C468201D00F0DAFB94F828005A
:1064D00000F00400E8B1A06941192B463A46204675
:1064E000FFF7A2FFD8B1002003462A4601460090DC
:1064F000204601F063FD064656B900BF502080F3E8
:106500001188BFF34F8FBFF36F8F00BF00BFFEE74F
:1065100005E094F8280020F0010084F828002046C7
:10652000216A8847F8BD000080000020F0B587B0E0
:10653000A0E00398002811DA04AE56B900BF50203D
:1065400080F31188BFF34F8FBFF36F8F00BF00BF81
:10655000FEE7D6E90020B168904700BF0398002805
:10656000E6DB059C606908B9012000E0002010B955
:10657000201D00F085FB02A800F0DEF80546039818
:106580000A2875D2DFE800F00905073941630608DB
:106590003A4200BF00BF00BF00BF94F8280040F09F
:1065A000010084F828000498A269811803462A464D
:1065B0002046FFF739FFF8B12046216A884794F852
:1065C000280000F00400B8B1002000900498A169F0
:1065D000421800231946204601F0F0FC074657B93F
:1065E00000BF502080F31188BFF34F8FBFF36F8F30
:1065F00000BF00BFFEE700BF3BE000BF94F82800EB
:1066000020F0010084F8280033E000BF94F828004F
:1066100040F0010084F828000498A061A06908B146
:10662000012000E0002050B900BF502080F3118805
:10663000BFF34F8FBFF36F8F00BF00BFFEE7A069AE
:1066400041192B462A462046FFF7EEFE11E094F84A
:10665000280000F0020018B9204600F0CFFB05E04A
:1066600094F8280020F0010084F8280001E0FFE7FA
:1066700000BF00BF002203A90448006801F0ACF885
:1066800000287FF456AF07B0F0BD0000880000205E
:10669000F8B505460C4600F067FD684600F04CF87A
:1066A0000646009820BB44B9B54206D801F074FBF9
:1066B00031462846FFF700FF1CE03CB10E48006859
:1066C000006808B9012000E000200446A91B22460A
:1066D0000A48006800F04AFC01F05EFB50B94FF038
:1066E000805007490860BFF34F8FBFF36F8F01E001
:1066F00001F052FBF8BD000084000020880000205B
:1067000004ED00E00A490968096809B9012100E0BF
:10671000002121B14FF0FF31064A116006E0044923
:106720000968C968C868034A416811607047000079
:10673000480000207400002070B5044601F0E6F91E
:10674000054607480068854204D200F00BF8012096
:10675000206001E00020206001480560284670BDEF
:10676000900000202DE9F84334E025480068C06817
:10677000056823480068C068C468201D00F080FADE
:106780002046216A884794F8280000F0040008B3E6
:10679000A0694619AE4207D966602461211D1848D8
:1067A000006800F0BDFA15E0002003462A460146C5
:1067B0000090204601F002FC074657B900BF502068
:1067C00080F31188BFF34F8FBFF36F8F00BF00BFFF
:1067D000FEE700BF0A480068006808B9012000E031
:1067E00000200028C1D00648D0F800800548006885
:1067F000034908600348C0F80080BDE8F883000042
:1068000080000020840000200246002101E0521C8C
:10681000491C1078A528FAD0890888B27047000072
:106820000E480068401C08B9012000E0002050B963
:1068300000BF502080F31188BFF34F8FBFF36F8FDD
:1068400000BF00BFFEE700BF502080F31188BFF3F8
:106850004F8FBFF36F8F00BF00BFFEE7B80000206F
:1068600008B500BF6846FFF76FFC04462046009954
:10687000FFF70EFFFFF75AFEF4E770B5044600F08D
:1068800075FA94F9455010E0606A08B9012000E0FB
:10689000002038B904F1240001F032FA18B100F0F8
:1068A000C5FB00E003E0681E45B2002DECDC00BF34
:1068B000FF2084F8450000F083FA00F057FA94F9BD
:1068C000445010E0206908B9012000E0002048B9D8
:1068D00004F1100001F014FA08B100F0A7FB681EE3
:1068E00045B200E001E0002DECDC00BFFF2084F8A1
:1068F000440000F065FA70BD2DE9F04104464FF008
:10690000000800F031FC4948006808B9FFF730FC86
:10691000474800682040002870D1D4B1083404F002
:106920000700B0B104F00700C0F10800044404F00F
:10693000070008B9012000E0002050B900BF502036
:1069400080F31188BFF34F8FBFF36F8F00BF00BF7D
:10695000FEE7002C52D03748006884424ED8364EAD
:106960003046056801E02E462D686868A04202D2D4
:1069700028680028F7D12D48006885423ED030684D
:1069800000F10808286830606868001B102819D9D1
:106990002F1907F0070008B9012000E0002050B9C6
:1069A00000BF502080F31188BFF34F8FBFF36F8F6C
:1069B00000BF00BFFEE76868001B78606C60384667
:1069C000FFF7FEFC1B4968680968081A1949086046
:1069D0000846006819490968884203D215480068CA
:1069E0001649086012496868096808436860002011
:1069F000286013480068401C1149086001F0CCF978
:106A000008F0070008B9012000E0002050B900BFDD
:106A1000502080F31188BFF34F8FBFF36F8F00BFFB
:106A200000BFFEE74046BDE8F0810000A000002066
:106A3000B4000020A400002098000020A80000203E
:106A4000AC00002070B50446254654B900BF502064
:106A500080F31188BFF34F8FBFF36F8F00BF00BF6C
:106A6000FEE700F083F9EE6900F0AAF9304670BD48
:106A7000001F4FF080730360001F21F001030360CB
:106A8000001F054B036014380260001F6FF0020303
:106A900003602038704700002168000810B52948BD
:106AA000008828494988884200D110BD254841887E
:106AB000001D405C0F283BD1224840881830C0F3AD
:106AC00008012048001D405C88BB1E4840881730E4
:106AD000C0F308011B48001D405C40BB19480088FA
:106AE00018494988401AC0F30800192827DB0024F8
:106AF0000BE0144840882044C0F308011148001DF1
:106B0000405C11490855601CC4B2192CF1DB0E48D9
:106B100000F01CF8FDF7E6F80A4840881930C0F389
:106B20000800084948800020A1F8060207E0FFE7B6
:106B300004484088401CC0F308000249488000BF58
:106B4000B3E7000064090020A00F0020417882789C
:106B500041EA0221C1F30A01484A11808178C91033
:106B6000C27841EA4211C1F30A01444A5180C17816
:106B70008911027941EA8201427941EA8221C1F315
:106B80000A013E4A918041794910827941EAC21155
:106B9000C1F30A01394AD18081790911C27941EAE8
:106BA0000211C1F30A01354A1181C179C911027A72
:106BB00041EA4201427A41EA4221C1F30A012F4AE5
:106BC0005181417A8910827A41EA8211C1F30A0126
:106BD0002A4A9181817A4911C27A41EAC201274A3F
:106BE000D181017B427B41EA0221C1F30A01234AA0
:106BF0001182417BC910827B41EA4211C1F30A0133
:106C00001E4A5182817B8911C27B41EA8201027C4A
:106C100041EA8221C1F30A01184A9182017C49109C
:106C2000427C41EAC211C1F30A01144AD182417C7B
:106C30000911827C41EA0211C1F30A010F4A118352
:106C4000817CC911C27C41EA4201027D41EA4221B4
:106C5000C1F30A01094A5183017D8910427D41EA4D
:106C60008211C1F30A01054A9183417D4911827D58
:106C700041EAC201014AD18370470000BA0F0020E7
:106C800001460A69D1E901309860D1E901035860F1
:106C90005068884201D188685060002008611068FF
:106CA000401E1060106870472DE9F041044614B989
:106CB0000648006800E0204607463D6B2846FFF77F
:106CC000A3FD06463046BDE8F081000044000020E8
:106CD000034B0360034B0B604FF4807313607047EA
:106CE000F815002054160020034B0360034B0B6083
:106CF0004FF4007313607047541A0020B01A00203C
:106D000000F1080141604FF0FF31816000F108019E
:106D1000C16001610021016070470021016170477D
:106D200010B502460B685C1C0CB9106907E002F153
:106D3000080000E04068446824689C42FAD944682E
:106D40004C604C68A160886041600A611468641CF2
:106D5000146010BD42684A6093688B609368596004
:106D60009160086103685B1C0360704700BF50209E
:106D700080F31188BFF34F8FBFF36F8F00BF0E48B2
:106D80000068401C0C49086008460068012812D1C0
:106D90000A480068C0B208B9012000E0002050B9DC
:106DA00000BF502080F31188BFF34F8FBFF36F8F68
:106DB00000BF00BFFEE77047B800002004ED00E010
:106DC0000D48006850B900BF502080F31188BFF310
:106DD0004F8FBFF36F8F00BF00BFFEE7064800680C
:106DE000401E054908600846006820B9002080F36D
:106DF000118800BF00BF7047B800002070B506467C
:106E00003546002E44D0083D2C462249606809686A
:106E1000084008B1012000E0002050B900BF502018
:106E200080F31188BFF34F8FBFF36F8F00BF00BF98
:106E3000FEE7206808B9012000E0002050B900BF3B
:106E4000502080F31188BFF34F8FBFF36F8F00BFC7
:106E500000BFFEE70F49606809680840C0B12068BC
:106E6000B0B90C49606809688843606000F07CF93B
:106E70000949606809680844074908602046FFF727
:106E80009FFA06480068401C0449086000F084FF2F
:106E900070BD0000B4000020A4000020B00000205D
:106EA00000204FF0E02108618861064800684FF437
:106EB0007A71B0FBF1F0401E4FF0E02148610720ED
:106EC000086170474000002070B5F9F7C3F9044627
:106ED000102C16D304F1E02090F8F05315480078F8
:106EE000854201DB012000E0002050B900BF5020A6
:106EF00080F31188BFF34F8FBFF36F8F00BF00BFC8
:106F0000FEE70D48006800F4E0600C49096888421B
:106F100001D8012000E0002050B900BF502080F3CC
:106F20001188BFF34F8FBFF36F8F00BF00BFFEE725
:106F300070BD0000BC0000200CED00E0C00000208F
:106F4000024600200BE0084B53F8303033B9064BB3
:106F500043F8301003EBC0035A6002E0401C0828DD
:106F6000F1D300BF70470000DC0F00202DE9F04195
:106F700005460E4617462C46FFF7F8FE94F94400E6
:106F8000401C10B9002084F8440094F94500401CCE
:106F900010B9002084F84500FFF712FFA06B28B954
:106FA0003A46314604F1240000F062F82046FFF72B
:106FB00064FCBDE8F081000070B504460025D4B142
:106FC0001248006808B9012000E0002050B900BF55
:106FD000502080F31188BFF34F8FBFF36F8F00BF36
:106FE00000BFFEE700F0C0F800212046FEF738FFA2
:106FF00000F0D2FE05463DB94FF0805004490860CC
:10700000BFF34F8FBFF36F8F70BD00007C00002077
:1070100004ED00E003490968016003490968416023
:10702000704700006C00002058000020012001493A
:10703000086070476800002070B504460D4654B9DA
:1070400000BF502080F31188BFF34F8FBFF36F8FC5
:1070500000BF00BFFEE70548016818312046FFF772
:107060005FFE01212846FEF7FBFE70BD44000020B4
:1070700070B505460E46144655B900BF502080F342
:107080001188BFF34F8FBFF36F8F00BF00BFFEE7C4
:107090000648016818312846FFF75CFE0CB14FF036
:1070A000FF3621463046FEF7DBFE70BD440000206F
:1070B00010B586B000200590049003AA04A905A885
:1070C000FFF706FE0022DDE904101346CDE900219A
:1070D00002901EA11F48039A00F0AAFC1E490860F6
:1070E0000846006808B1012400E00024012C02D108
:1070F00000F028FF0446012C15D100BF502080F37A
:107100001188BFF34F8FBFF36F8F00BF4FF0FF3079
:1071100012490860012012490860002011490860E6
:1071200000F07EF810E0601C08B1012000E00020B3
:1071300050B900BF502080F31188BFF34F8FBFF3C9
:107140006F8F00BF00BFFEE706B010BD49444C453D
:1071500000000000ED6100087800002074000020AD
:10716000600000205800002002480068401C0149CF
:10717000086070477C0000201E48006818B101209C
:107180001D49086034E000201B4908601B48016865
:107190000CE051B900BF502080F31188BFF34F8F2E
:1071A000BFF36F8F00BF00BFFEE7491E01EB8100F8
:1071B000134A52F8200008B9012000E000200028FE
:1071C000E7D101EB81020E4B03EB8200426852686B
:1071D000426000F108024368934202D1426852685B
:1071E00042604268D268074B1A600448016000BFE1
:1071F000704700007C000020680000205C00002038
:107200001C10002044000020014800687047000066
:10721000A40000200148006870470000A80000207A
:107220001CB5524800685249884201D0012000E054
:10723000002050B900BF502080F31188BFF34F8F5A
:10724000BFF36F8F00BF00BFFEE7484800684849A2
:10725000491E884201D0012000E0002050B900BF43
:10726000502080F31188BFF34F8FBFF36F8F00BFA3
:1072700000BFFEE73F49084600780190FF200A461C
:1072800010700846007800909DF8000000F0F000B3
:107290009DF80020904201D1012000E0002050B96B
:1072A00000BF502080F31188BFF34F8FBFF36F8F63
:1072B00000BF00BFFEE79DF8000000F050002E4A1E
:1072C000107007202D4A106009E02C480068401E0D
:1072D0002A4A10609DF800004006000E00909DF8BC
:1072E000000000F080008028EFD024480068C0F142
:1072F0000700042801D1012000E0002050B900BFA0
:10730000502080F31188BFF34F8FBFF36F8F00BF02
:1073100000BFFEE7194800680002184A10601046D6
:10732000008800F4E0601060124A019810700F4865
:107330002030006840F470000C4920310860084695
:10734000006840F070400860FFF7AAFD00200C497B
:107350000860F8F747FF0B48006840F040400949D3
:107360000860F8F72BFF00201CBD000000ED00E0D6
:1073700071C20F4100E400E0BC000020C00000200A
:10738000B800002034EF00E010B500BF502080F3BB
:107390001188BFF34F8FBFF36F8F00BF00F0BCFBAE
:1073A00018B14FF080500449086000BF002080F3FE
:1073B000118800BF10BD000004ED00E02DE9F84386
:1073C00080460E4617461D46DDF82090B8F1000FA6
:1073D00001D0012000E0002050B900BF502080F310
:1073E0001188BFF34F8FBFF36F8F00BF00BFFEE761
:1073F0000DB1012000E0002050B900BF502080F303
:107400001188BFF34F8FBFF36F8F00BF00BFFEE740
:1074100007B10EB1012000E0002050B900BF50209C
:1074200080F31188BFF34F8FBFF36F8F00BF00BF92
:10743000FEE707B90EB9012000E0002050B900BFF7
:10744000502080F31188BFF34F8FBFF36F8F00BFC1
:1074500000BFFEE7502000900098502801D1012085
:1074600000E0002050B900BF502080F31188BFF326
:107470004F8FBFF36F8F00BF00BFFEE700BF2C46EA
:107480004CB1012084F846004B463A46314640460E
:107490000094FEF7BFFE2046BDE8F88370B50546B0
:1074A0000E462C4654B900BF502080F31188BFF31C
:1074B0004F8FBFF36F8F00BF00BFFEE7FFF756FC93
:1074C000D4E90F12206801FB0200A0600020A06335
:1074D00020686060E06B401E226C216800FB021196
:1074E000E160FF2084F8440084F845009EB92069DB
:1074F00008B9012000E00020A8B904F1100000F054
:10750000FFFB80B14FF0805009490860BFF34F8FF7
:10751000BFF36F8F07E004F11000FFF7F1FB04F1F8
:107520002400FFF7EDFBFFF74BFC012070BD0000CE
:1075300004ED00E02DE9FF4383B0064688461D4672
:107540004FF00009344654B900BF502080F3118831
:10755000BFF34F8FBFF36F8F00BF00BFFEE7B8F1DF
:10756000000F01D1206C08B9012000E0002050B9C3
:1075700000BF502080F31188BFF34F8FBFF36F8F90
:1075800000BF00BFFEE7022D02D1E06B012801D150
:10759000012000E0002050B900BF502080F3118886
:1075A000BFF34F8FBFF36F8F00BF00BFFEE700F048
:1075B0009DFA08B9059808B9012000E0002050B9EB
:1075C00000BF502080F31188BFF34F8FBFF36F8F40
:1075D00000BF00BFFEE700BFFFF7C8FBA06BE16B79
:1075E000884201D3022D28D12A4641462046FEF783
:1075F00044FD0746606A08B9012000E0002068B930
:1076000004F1240000F07CFB88B14FF08050324937
:107610000860BFF34F8FBFF36F8F08E03FB14FF0AB
:1076200080502D490860BFF34F8FBFF36F8FFFF776
:10763000C7FB012007B0BDE8F083059818B9FFF734
:10764000BFFB0020F6E7B9F1000F04D101A8FFF756
:10765000E1FC4FF00109FFF7B3FBFFF785FDFFF7F2
:1076600085FB94F94400401C10B9002084F84400C4
:1076700094F94500401C10B9002084F84500FFF73C
:107680009FFB05A901A800F05BF9F0B92046FEF7C1
:1076900004FFA0B104F110000599FFF7CDFC2046CE
:1076A000FFF7EBF800F078FB002895D14FF0805001
:1076B00009490860BFF34F8FBFF36F8F8CE72046F7
:1076C000FFF7DBF800F068FB86E72046FFF7D5F808
:1076D00000F062FB0020ADE704ED00E02DE9F84F7B
:1076E00007468A4690461E463C4654B900BF502085
:1076F00080F31188BFF34F8FBFF36F8F00BF00BFC0
:10770000FEE7BAF1000F01D1206C08B9012000E0BA
:10771000002050B900BF502080F31188BFF34F8F75
:10772000BFF36F8F00BF00BFFEE7022E02D1E06BF8
:10773000012801D1012000E0002050B900BF5020F5
:1077400080F31188BFF34F8FBFF36F8F00BF00BF6F
:10775000FEE7FFF7B9FB00BF5021EFF3118081F383
:107760001188BFF34F8FBFF36F8F00BF0546A06B2B
:10777000E16B884201D3022E25D194F945B0A06B6C
:107780000090324651462046FEF777FC0BF101008F
:1077900088B9606A08B9012000E0002050B904F1FE
:1077A000240000F0ADFA28B1B8F1000F02D001209A
:1077B000C8F8000004E00BF1010040B284F8450075
:1077C0004FF0010901E04FF0000900BF85F3118877
:1077D00000BF4846BDE8F88F2DE9F74183B0054664
:1077E0000E464FF000082C4654B900BF502080F3DD
:1077F0001188BFF34F8FBFF36F8F00BF00BFFEE74D
:107800000EB9206C08B9012000E0002050B900BF7B
:10781000502080F31188BFF34F8FBFF36F8F00BFED
:1078200000BFFEE700F062F908B9059808B9012029
:1078300000E0002050B900BF502080F31188BFF352
:107840004F8FBFF36F8F00BF00BFFEE700BFFFF792
:107850008DFAA76BF7B131462046FEF7F9FB781E8B
:10786000A063206908B9012000E0002060B904F19C
:10787000100000F045FA38B14FF080502F490860F1
:10788000BFF34F8FBFF36F8FFFF79AFA012006B057
:10789000BDE8F081059818B9FFF792FA0020F6E7E5
:1078A000B8F1000F04D101A8FFF7B4FB4FF00108B5
:1078B000FFF786FAFFF758FCFFF758FA94F94400EF
:1078C000401C10B9002084F8440094F94500401C85
:1078D00010B9002084F84500FFF772FA05A901A845
:1078E00000F02EF8F0B92046FEF7CAFDA0B104F171
:1078F00024000599FFF7A0FB2046FEF7BEFF00F02D
:107900004BFA0028A3D14FF080500C490860BFF318
:107910004F8FBFF36F8F9AE72046FEF7AEFF00F060
:107920003BFA94E72046FEF7A8FF00F035FA204620
:10793000FEF7A6FD00288AD00020A8E704ED00E0AD
:1079400070B505460C4655B900BF502080F311882C
:10795000BFF34F8FBFF36F8F00BF00BFFEE754B977
:1079600000BF502080F31188BFF34F8FBFF36F8F9C
:1079700000BF00BFFEE7FFF7F9F912480268686828
:10798000131A2068401C08B9002617E00E49286821
:107990000968884204D06868904201D801260DE049
:1079A0002068984207D92068C01A20602846FFF74F
:1079B00031FB002602E0002020600126FFF700FADC
:1079C000304670BD580000206C0000202DE9FF4FAC
:1079D00085B0804689461746DDE912ABB800FEF750
:1079E0008BFF064656B15C20FEF786FF04460CB1BD
:1079F000266304E03046FFF701FA00E000248CB172
:107A0000002084F85900CDE900ABCDE902403A46A8
:107A100049464046089BFEF712FC2046FEF75EFAF8
:107A2000012501E04FF0FF35284609B0BDE8F08F91
:107A30002DE9F04F85B00746884691469A46DDE924
:107A40000EB6109C0EB1012000E0002050B900BF1E
:107A5000502080F31188BFF34F8FBFF36F8F00BFAB
:107A600000BFFEE70CB1012000E0002050B900BFCC
:107A7000502080F31188BFF34F8FBFF36F8F00BF8B
:107A800000BFFEE75C20039003985C2801D1012031
:107A900000E0002050B900BF502080F31188BFF3F0
:107AA0004F8FBFF36F8F00BF00BFFEE700BFB4B1C1
:107AB000AEB125462C462E63022085F859000020E1
:107AC00004A953464A46CDE900B1CDE902504146EA
:107AD0003846FEF7B4FB2846FEF700FA01E0002026
:107AE0000490049805B0BDE8F08F000005490968CE
:107AF00009B9012005E00449096809B9022000E03C
:107B000000207047600000207C00002001490868C8
:107B100070470000580000202DE9F0414FF00008A8
:107B20004348006800287BD142480068451C414812
:107B3000056015BB40480068006808B9012000E0F6
:107B4000002050B900BF502080F31188BFF34F8F41
:107B5000BFF36F8F00BF00BFFEE7374807683748A5
:107B60000068354908603548076035480068401CA2
:107B700033490860FEF7C6FD00BF32480068854201
:107B80003BD300BF2C480068006808B9012000E022
:107B9000002020B14FF0FF302A4908602CE0264831
:107BA0000068C068C4686668B54202D225480660AD
:107BB00022E0201DFFF764F8A06A18B104F1180054
:107BC000FFF75EF82049E06A0968884202D91E4939
:107BD000E06A0860E16A01EB81011C4A02EB810066
:107BE000211DFFF7B7F81A49E06A0968C96A884297
:107BF000C8D34FF00108C5E700BF15480068C06A48
:107C000000EB8000114951F82000012801D94FF004
:107C100001081048006808B14FF0010805E0FFE7CF
:107C20000D480068401C0C4908604046BDE8F081E2
:107C30007C00002058000020480000204C0000205C
:107C40006C000020740000205C0000201C1000204C
:107C500044000020680000206400002070B5054644
:107C60002C460026002D43D022480068844201D1D2
:107C7000012000E0002050B900BF502080F311889F
:107C8000BFF34F8FBFF36F8F00BF00BFFEE7206DC4
:107C900050B900BF502080F31188BFF34F8FBFF35E
:107CA0006F8F00BF00BFFEE7206D401E2065E16CB6
:107CB000E06A88421CD0206DD0B9201DFEF7E0FF9D
:107CC000E06CE062E06AC0F13800A0610A49E06A55
:107CD0000968884202D90849E06A0860E16A01EB54
:107CE0008101064A02EB8100211DFFF733F80126CE
:107CF000304670BD440000205C0000201C100020B5
:107D000070B50646F068C46854B900BF502080F3CF
:107D10001188BFF34F8FBFF36F8F00BF00BFFEE727
:107D200004F11800FEF7ACFF15480068A0B9201D4B
:107D3000FEF7A6FF1349E06A0968884202D9114993
:107D4000E06A0860E16A01EB81010F4A02EB810001
:107D5000211DFEF7FFFF04E004F118010B48FEF7B8
:107D6000F9FF0B49E06A0968C96A884204D901250C
:107D700001200849086000E00025284670BD000089
:107D80007C0000205C0000201C100020A4140020B7
:107D9000440000206800002070B50024002636480A
:107DA000006850B900BF502080F31188BFF34F8F97
:107DB000BFF36F8F00BF00BFFEE7FEF7D7FF2E486F
:107DC0000068401E2C4908600846006800284ED113
:107DD0002A48006800284AD023E02948C068C468BF
:107DE00004F11800FEF74CFF201DFEF749FF25495E
:107DF000E06A0968884202D92249E06A0860E16ABB
:107E000001EB8101204A02EB8100211DFEF7A2FF58
:107E10001E49E06A0968C96A884202D301201C49E8
:107E200008601748006808B9012000E00020002819
:107E3000D3D00CB1FEF766FC1648056865B100BFEB
:107E4000FFF76AFE10B10120114908606D1E002D78
:107E5000F6D100200F4908600D48006838B10126AE
:107E600030070D490860BFF34F8FBFF36F8FFEF7E8
:107E7000A7FF304670BD00007C00002054000020A9
:107E8000A41400205C0000201C10002044000020EE
:107E9000680000206400002004ED00E02DE9FC47AC
:107EA00005460E4617469846DDF828902C20FEF72A
:107EB00023FD044654B1002084F8280043463A4686
:107EC00031462846CDE90094FEF718FA2046BDE871
:107ED000FC872DE9FC4706460F4690469946DDE9AA
:107EE0000AA52C20019001982C2801D1012000E046
:107EF000002050B900BF502080F31188BFF34F8F8E
:107F0000BFF36F8F00BF00BFFEE700BF55B900BFD2
:107F1000502080F31188BFF34F8FBFF36F8F00BFE6
:107F200000BFFEE72C4654B1022084F828004B46DF
:107F3000424639463046CDE900A4FEF7DFF9204637
:107F4000BDE8FC8710B586B00024FEF723F816487C
:107F50000068D0B100200590049003AA04A905A8E8
:107F6000FEF7C2FE0222DDE904100023CDE9002164
:107F700002900EA10F48039AFFF75AFD0E490860C0
:107F80000846006800B1012400BF54B900BF50206A
:107F900080F31188BFF34F8FBFF36F8F00BF00BF17
:107FA000FEE7204606B010BD88000020546D722008
:107FB00053766300616800088C0000202DE9FF47BC
:107FC00004460D4616461F46DDF830804FF0000986
:107FD00054B900BF502080F31188BFF34F8FBFF317
:107FE0006F8F00BF00BFFEE71448006810B3009514
:107FF00001960294062D15DAFFF778FD022808D1C4
:108000000023424669460D480068FFF793FA81460F
:1080100010E000231A46694608480068FFF78AFA0C
:10802000814607E000233A46694604480068FFF7A6
:1080300055FB8146484604B0BDE8F0878800002023
:108040003481000800000000000000000000000073
:1080500000000000000800002800000000000000F0
:10806000000000001C81000800000000000000006B
:1080700000000000000000000008000020000000D8
:10808000000000000000000028810008000000003F
:1080900000000000000000000000000000080000D8
:1080A0001000000000000000000000001081000827
:1080B0000000000000000000000000000006101694
:1080C000000610160000000000000000010203047A
:1080D00006070809000000000102030430313233B2
:1080E00034353637383941424344454600000000B4
:1080F0000000545452205245474745530030313216
:108100003334353637383941424344454600000060
:108110006D7954696D657230310000006D7954617C
:10812000736B3032000000006D795461736B303333
:108130000000000064656661756C745461736B00C7
:108140006081000800000020C4000000BA5A000846
:1081500024820008C4000020A4F20000CA5A0008CB
:10816000000000000000000000000000000000000F
:1081700000000000000000000000000000000000FF
:1081800000000000000000000000000000000000EF
:10819000F4010000000000001000000001000000D9
:1081A0000024F400000000000000000000000000B7
:1081B00000000000000000000000000000000000BF
:1081C00000000000000000000000000000000000AF
:1081D000000000000000000000000000000000009F
:1081E000000000000000000000000000000000008F
:1081F000000000000000000000000000000000007F
:10820000000000000000000000000000000000006E
:108210000000000000000000AAAAAAAA00000000B6
:04822000000000005A
:040000050800018965
:00000001FF
